:1000000053C6000070C600006EC600006CC600003B
:100010006AC6000068C6000066C6000064C600002C
:1000200062C600000C941F195EC600000C94CF1825
:100030005BC6000058C600000C94F71854C60000B8
:100040000C94A71850C600004EC600004CC6000015
:100050004AC600000C944E1946C6000044C6000073
:1000600042C6000040C600003EC600003CC600007C
:100070003AC6000038C6000036C6000034C600008C
:1000800032C6000030C600002EC600000B120D1252
:100090000D1210121012101210121012131215124B
:1000A0001512151215122D123112092184213C202E
:1000B0008B1F4A236A213C2278229C226C249226A0
:1000C00071278A27E427722AEB281F292929422928
:1000D0005F29322A412A722A782A8F2BBD2BF325D9
:1000E00012260B260B26F625F925FC250B260B26BA
:1000F0000B260B26FF2502260B2605260826852C17
:10010000E92C0B2CF42B9D2EE62C722E762E8A2EAB
:100110004B30442F2C306830773128322F32A233C5
:1001200081328432A932A233B832E3321833F73243
:10013000BF2EC82ECF2ED62EDD2EF12EFF2E0B2F4A
:10014000152FAA345F34AC34AC34AC347434AC34D2
:10015000AC349734AC34AA34AA34AC34AC34AC34B8
:10016000AC34AC34AC34AC34AC34AC344F34573441
:100170002F5341564553001F1C1F1E1F1E1F1F1EBD
:100180001F1E1F10278813D007E803E803E803F4B5
:1001900001F401320032003200320081008000425E
:1001A000415700544150002E424157002E574156AE
:1001B000002E54415000EFEEE6E0EBF3E9F1F2E0FF
:1001C0002E2E00776169742E2E2E00CFEEE4EEE61F
:1001D000E4E8F2E500506C656173650020EEF8E834
:1001E000E1EEEA00206572726F727300D2E0E9EC12
:1001F000E0F3F220E7E0EFE8F1E800577269746598
:100200002074696D656F757400D2E0E9ECE0F3F27B
:1002100020F7F2E5EDE8FF00526561642074696D36
:10022000656F757400D2E0E9ECE0F3F220522F57CD
:1002300000522F572074696D656F757400C7E0E335
:10024000F0F3E7EAE000506C6179696E6700D1CEA7
:10025000D5D0C0CDC8D2DC20CAC0CA005341564553
:1002600020415300EAE0F0F2F320EFE0ECFFF2E887
:100270000053442D4341524400C2F1F2E0E2FCF24B
:10028000E500496E7365727400F4E0E9EBE0006626
:100290006F726D617400CDE5E2E5F0EDFBE920F4ED
:1002A000EEF0ECE0F20057726F6E672066696C65E5
:1002B00000F4E0E9EB0066696C6500CDE520ECEE4A
:1002C000E3F320F1EEF5F0E0EDE8F2FC0043616EBF
:1002D000277420777269746500F4E0E9EB006669C1
:1002E0006C6500CDE520ECEEE3F320EFF0EEF7E8EF
:1002F000F2E0F2FC0043616E2774207265616400D5
:10030000F4E0E9EB0066696C6500CDE520ECEEE316
:10031000F320F1EEE7E4E0F2FC0043616E27742085
:1003200063726561746500CED8C8C1CAC000455209
:10033000524F5200CAEEEDF2F0E0F1F2EDEEF1F2C2
:10034000FC00436F6E747261737400C7E0ECE5EDFE
:10035000E8F2FC20E5E3EE3F005265706C616365F6
:100360002069743F00D3E6E520F1F3F9E5F1F2E20C
:10037000F3E5F200416C7265616479206578697318
:10038000747300D1E5EAF2EEF03A2000536563742D
:100390006F723A2000CAEBE0F1F2E5F03A20004338
:1003A0006C75737465723A2000D0E0E7ECE5F0FB01
:1003B0000053697A657300D0E0E7E4E5EB00506133
:1003C00072746974696F6E3A00455854454E4445DD
:1003D00044204C4241004641543136204C424100B9
:1003E0004641543332204C4241004641543332009E
:1003F000464154313600457874656E646564004644
:1004000041543136202833324D622900464154315F
:10041000320046726565002000290028002F004B3D
:1004200000CCE1004D4200CDE5E8E7E2E5F1F2E580
:10043000ED00556E6B6E6F776E00D3EDE8E2E5F080
:10044000F1E0EBFCEDFBE900556E697665727361D6
:100450006C005375706572466C6F707079004861FE
:1004600072644469736B20284D42522900D4EEF027
:10047000ECE0F23A00466F726D61743A00D0E5E24A
:10048000E8E7E8FF3A20005265766973696F6E3AD3
:100490002000C8ECFF20EFF0EEE4F3EAF2E03A00CF
:1004A00050726F64756374206E616D653A00CEE1C1
:1004B000FAE5EC0053697A6500D1E5F02E20EDEE07
:1004C000ECE5F00053657269616C206E756D6265D4
:1004D0007200CFF0EEE8E7E2EEE4E8F2E5EBFC00D4
:1004E0004D616E75666163747572657200D1E2EE7E
:1004F000E1EEE4EDEE2C20CCE100467265652C20A7
:100500004D4200C1EBEEEAE83A00426C6F636B7358
:100510003A00E1E0E9F200627974657300E100629B
:1005200000EFE8EBEEF20070696C6F74007777779C
:100530002E74726F6C736F66742E72750032303168
:10054000350085864F6C656720547269666F6E6FE3
:100550007600762E20312E31005A58205461706575
:100560007200F1E8E3EDE0EBE02E2E2E00746865FA
:10057000207369676E616C2E2E00CEE6E8E4E0ED34
:10058000E8E50057616974696E6720666F7200ED77
:10059000E0F1F2F0EEE9EAE83F00746F206465668E
:1005A00061756C743F00D1E1F0EEF1E8F2FC0052AD
:1005B000657365742073657474696E677300CFEE3C
:1005C00020F3ECEEEBF7E0EDE8FE004465666175C4
:1005D0006C7400CEEFF0E5E4E5EBE8F2FC00446576
:1005E0007465637400C7E0F5E2E0F2004361707483
:1005F00075726500C4E0EDEDFBE5004461746100D7
:10060000D1E8EDF52E320053796E63203200D1E847
:10061000EDF52E310053796E63203100CFE8EBEE1B
:10062000F20050696C6F7400CFE8EBEEF22EE4003C
:1006300050696C6F742E6C00ECEAF100757300EC7D
:10064000F1006D7300F4F0EEEDF200726973650075
:10065000F1EFE0E40066616C6C00D0F3F1005275DC
:100660007300C0EDE300456E670078380078340011
:10067000783200783100C0E2F2EE004175746F000C
:10068000C2FBEA004F666600C2EAEB004F6E00CA8A
:10069000EEEDF2F0E0F1F200D16F6E7472617374FE
:1006A00000C4E0F2E020E820E2F0E5ECFF00446165
:1006B000746520262074696D6500D2E0E9ECE8EDF0
:1006C000E3E80054696D696E677300D1EAEEF0EEFD
:1006D000F1F2FC00537065656400CFEEE4F1E2E5F1
:1006E000F2EAE000486967686C6967687400C7E20D
:1006F000F3EA20E7E0EF2E00536F756E6420726519
:100700006300C7E2F3EA20E2F1EFF02E00536F75C9
:100710006E6420706C617900C7E2F3EA20EAEBE0D6
:10072000E22E00536F756E64206B657900DFE7FB86
:10073000EA004C616E677561676500C8CDD4CE0074
:1007400041424F555400534420CAC0D0D2C0005338
:100750004420494E464F00CDC0D1D2D0CEC9CAC8E0
:100760000053455454494E475300D1CED5D0C0CD47
:10077000C8D2DC005341564500CFD0CED7C8D2C036
:10078000D2DC00504C415900C7E0E3F0F3E7EAE067
:100790002E2E2E004C6F6164696E672E2E2E00C3C4
:1007A000EEF2EEE2EE00446F6E65003CCFF3F1F244
:1007B000EE3E003C456D7074793E00CEF8E8E1EA0B
:1007C000E02043524300435243206572726F72002F
:1007D000D4E0E9EB20EFEEE2F0E5E6E4E5ED210020
:1007E00046696C652062726F6B656E2100C1EBEE2D
:1007F000EA00426C6F636B00CDE0E7E0E400426129
:10080000636B00CDE5F2004E6F00C4E000596573E4
:1008100000CEF2ECE5EDE00043616E63656C00CF65
:10082000F0EEE4EEEBE6E8F2FC00526573756D6500
:1008300000CFE0F3E7E000506175736500D1F2EEA0
:10084000EF0053746F7000000000000000005F00B4
:10085000000007000700147F147F14242A7F2A1247
:100860002313086462364955225000050300000036
:100870001C2241000041221C00082A1C2A080808EA
:100880003E080800503000000808080808006060B2
:10089000000020100804023E5149453E00427F40BE
:1008A0000042615149462141454B311814127F10D5
:1008B00027454545393C4A49493001710905033608
:1008C00049494936064949291E0036360000005676
:1008D0003600000008142241141414141441221488
:1008E00008000201510906324979413E7E11111179
:1008F0007E7F494949363E414141227F4141221C88
:100900007F494949417F090901013E414151327FF7
:100910000808087F00417F41002040413F017F08D7
:100920001422417F404040407F0204027F7F040840
:10093000107F3E4141413E7F090909063E41512158
:100940005E7F09192946464949493101017F010164
:100950003F4040403F1F2040201F7F2018207F63E2
:1009600014081463030478040361514945430000EB
:100970007F4141020408102041417F000004020130
:1009800002044040404040000102040020545454FE
:10099000787F484444383844444420384444487FAD
:1009A0003854545418087E090102081454543C7FEA
:1009B0000804047800447D40002040443D00007F4E
:1009C00010284400417F40007C041804787C08040F
:1009D000047838444444387C141414080814141857
:1009E0007C7C080404084854545420043F444020AC
:1009F0003C4040207C1C2040201C3C4030403C447B
:100A0000281028440C5050503C4464544C44000876
:100A100036410000007F0000004136080008082A27
:100A20001C08081C2A08081436773614007F3E1C60
:100A300008081C3E7F0004060706041030703010C2
:100A40003E41081414413E00000010387C101F087D
:100A50001C3E08080000000000000000000000002C
:100A60000000000000000000000000000000000086
:100A70000000000000000000000000000000000076
:100A80000000000000000000000000000000000066
:100A90000000000000000000000000000000000056
:100AA0000000000000000000000000000000000046
:100AB0000000000000000000000000000000000036
:100AC0000000000000000000000000000000000026
:100AD0000000000000000000000000000000000016
:100AE0000000000000000000000000000000000006
:100AF00000000000000000000000000000000000F6
:100B000000000000000000000000000000000000E5
:100B100000000000000000000000000000000000D5
:100B200000000000000000000000000000000000C5
:100B300000000000000000000000000000000000B5
:100B400000000000000000000000000000000000A5
:100B50000000000000000000000000000000000095
:100B6000000000000000007E1111117E7F494949FC
:100B7000337F494949367F01010103E0514F41FF6D
:100B80007F4949494177087F087741494949367F7C
:100B90001008047F7C2112097C7F08142241204127
:100BA0003F017F7F020C027F7F0808087F3E4141A2
:100BB000413E7F0101017F7F090909063E41414114
:100BC0002201017F010147281008071C227F221CF7
:100BD00063140814637F404040FF070808087F7FC4
:100BE000407F407F7F407F40FF017F4848307F4803
:100BF00030007F007F484830224149493E7F083E0F
:100C0000413E462919097F20545454783C4A4A49A8
:100C1000317C545428007C0404040CE0544C44FC03
:100C200038545454186C107C106C44445454287C30
:100C30002010087C7C4122117C7C10284400204438
:100C40003C047C7C0810087C7C1010107C384444E8
:100C500044387C0404047C7C141414083844444450
:100C60002004047C04040C5050503C3048FC4830B4
:100C700044281028447C404040FC0C1010107C7C20
:100C8000407C407C7C407C40FC047C5050207C506C
:100C900050207C7C5050200028445454387C10381C
:100CA0004438085434147C0011241FBECFEFD0E127
:100CB000DEBFCDBF11E0A0E0B1E0EAECFCEB00E06C
:100CC0000BBF02C007900D92AE31B107D9F72EE0ED
:100CD000AEE1B1E001C01D92A435B207E1F70E9478
:100CE00062190C94635E8CC91F920F920FB60F921B
:100CF00011240BB60F928F939F93EF93FF93E09184
:100D00007605F09177050995FF91EF919F918F916D
:100D10000F900BBE0F900FBE0F901F9018950E9462
:100D200023520E941D528F930E941D52982F8F9123
:100D300008950E9423520E941D528F930E941D52BB
:100D40008F930E941D528F930E941D52982F8F9156
:100D50007F916F9108959F930E946B528F910C9495
:100D60006B529F938F93862F0E946B52872F0E9406
:100D70006B528F910E946B528F910C946B52F7E0E3
:100D8000E3EF9091F509E90FF11D80819395909320
:100D9000F50909F00895F6E0E5EEF093F409E09323
:100DA000F3090895FCE0E4E59091F509E90FF11DE0
:100DB000808193959093F50909F00895F6E0EDEFA1
:100DC000F093F409E093F3090895F8E0E3EF9091CC
:100DD000F509E90FF11D808193959093F50909F0CC
:100DE00008959091F6099E7F9093F609F7E0E5E368
:100DF000F093F409E093F3090895FDE0E4E59091A0
:100E0000F509E90FF11D808193959093F50909F09B
:100E100008959091F6099D7F9093F609F7E0E5E13A
:100E2000F093F409E093F30908958091F60980FFA7
:100E30000CC0F6E0EFEBF093F409E093F309809136
:100E4000F30791E09093F509089580913005816052
:100E50008093300580912E0590912F0501969093F7
:100E60002F0580932E0580E808958091F60981FF73
:100E70000CC0F6E0E2EDF093F409E093F309809101
:100E8000540C91E09093F5090895809130058160AC
:100E90008093300580912E0590912F0501969093B7
:100EA0002F0580932E0580E80895F7E0E3EF9091F9
:100EB000F509E90FF11D808393959093F50909F0E9
:100EC0000895F7E0EBE7F093530CE093520C08958C
:100ED000FCE0E4E59091F509E90FF11D808393951D
:100EE0009093F50909F00895F7E0E3E9F093530CC6
:100EF000E093520C0895F8E0E3EF9091F509E90FC3
:100F0000F11D808393959093F50909F008959091D0
:100F1000F60991609093F609F7E0EAECF093530C30
:100F2000E093520C0895FDE0E4E59091F509E90F96
:100F3000F11D808393959093F50909F008959091A0
:100F4000F60992609093F609F7E0EBEAF093530C00
:100F5000E093520C08959091F60990FF0FC0809194
:100F6000300582608093300580912E0590912F0589
:100F7000019690932F0580932E050895F7E0E5E5FF
:100F8000F093530CE093520C8093F30791E090930D
:100F9000F50908959091F60991FF0FC080913005F1
:100FA00082608093300580912E0590912F050196E7
:100FB00090932F0580932E050895F7E0E8E6F093CF
:100FC000530CE093520C8093540C91E09093F509EC
:100FD00008951DBC1CBCE091F309F091F40909953A
:100FE00087FF04C01B981092840008951B9A80917B
:100FF00007018093840008951DBC1CBC8091AC0740
:10100000811118C0E091F309F091F409099581115B
:1010100002C00C945C36982F9F779093AC0787FFA3
:1010200006C01B9A809107018093840003C01B981F
:10103000109284008091AC0781508093AC07089592
:1010400026B537B51DBC1CBC2F3F41E0340708F066
:10105000C2C036952795422F80910401813001F15D
:1010600020F0823009F456C0AAC081E080930401C8
:1010700080913F058F5F80933F058091400590915F
:1010800041059093430580934205109241051092CB
:10109000400582E10E946B5284E30E946B528FC034
:1010A00080914605811105C0273918F02093460527
:1010B00086C080914605882309F481C08091460549
:1010C0008695481708F07BC020933C0510921F01BD
:1010D00010921E0182E08093040180914705909157
:1010E0004805A0914905B0914A0520914B053091E2
:1010F0004C05820F931FA11DB11D8093470590934E
:101100004805A0934905B0934A0510924C051092EA
:101110004B0555C08091440581111BC083ED820FA2
:101120008A36B8F42A3518F42093440504C0822F77
:10113000869580934405C901880F991F63E070E08C
:101140000E94D95860933E05822F880F820F8093AA
:10115000450580913E05481790F18091450584171B
:1011600070F18091440543E0849FC001112495955E
:101170008795821793072CF480911F0181608093DB
:101180001F0180911E018F5F80931E01883090F0B7
:1011900080911F010E946B5280914B0590914C05EC
:1011A000019690934C0580934B0510921F0110926D
:1011B0001E0105C080911F01880F80931F012CB56F
:1011C0003DB580913D0590E08217930720F48CB5E2
:1011D0009DB580933D050895A4E0B0E0E2EFF8E00E
:1011E0000C94D75980910401813009F44AC08230AF
:1011F00009F04AC00E947152CE0101960E94EC5241
:101200008091470590914805A0914905B0914A0504
:1012100080914B0590914C05609147057091480570
:101220008091490590914A050E94FA5280914B05A0
:1012300090914C050E946B5280914B0590914C050A
:10124000892F0E946B520E94715269817A818B8131
:101250009C810E94FA528091470590914805A09187
:101260004905B0914A050296A11DB11D809347051D
:1012700090934805A0934905B0934A051092040144
:1012800003C083E0809304012496E2E00C94F359B8
:1012900080E791E00C9493510895EF92FF921F9391
:1012A000CF93DF9300D0CDB7DEB789839A83F0DF89
:1012B00089819A810E944554182F882309F46EC0B1
:1012C00010923F051092410510924005109243057F
:1012D000109242051FBC9EB593689EBD0E94891363
:1012E0009EB5813011F4906401C09F7B9EBD80E269
:1012F00086BF97B7946297BF10923D051092040184
:1013000010924705109248051092490510924A051F
:1013100010924C0510924B05109246051092440510
:101320000E9461137C010E940113970102C036954F
:1013300027958A95E2F7C9019695879596958795A1
:101340004FEF480F6AE070E00E94C558461B40937B
:1013500046050E947F137C010E940113F70102C021
:10136000F695E7958A95E2F7CF019695879596953C
:1013700087958093440520914405822F90E0880F43
:10138000991F63E070E00E94D95860933E058091F8
:101390004405982F990F980F90934505812F0F9032
:1013A0000F90DF91CF911F91FF90EF900895A4E0EF
:1013B000B0E0EDEDF9E00C94D75987B78B7D87BF8E
:1013C00084E0809304010E94D75269837A838B83DF
:1013D0009C830E94C55220913D0520914605209195
:1013E000460520913C0520913C0520914405209123
:1013F0004405209120013091210169817A818B81FE
:101400009C812496E2E00C94F3590E94C55287B760
:101410008B7D87BF84E0809304010895809104014F
:10142000823041F480914B0590914C059093410599
:10143000809340050E942B13882369F0809104015A
:10144000843049F0849B05C080910701809384001B
:1014500008951092840008958FE395E00895809197
:1014600004010895CF931DBC1CBC849B02C0C0E83E
:1014700001C0C0E080914D05C81313C08091AC0736
:101480008F5F8093AC078091AC078F37F8F0809125
:10149000AC0790914D05890F0E946B521092AC07DA
:1014A00015C08091AC0790914D05890F0E946B5239
:1014B000CC2329F0809107018093840002C0109210
:1014C0008400C0934D0581E08093AC07CF910895CF
:1014D000A2E0B0E0EEE6FAE00C94D65989839A8354
:1014E000D7DE89819A810E944554182F882309F1FB
:1014F00062E477E581E496E534DC81E090E02BDC82
:1015000084E49CEA28DC1092AC071FBC1DBC1CBC08
:101510002AE431E03BBD2ABD22E33AE0309377056F
:1015200020937605849B02C080E801C080E0809310
:101530004D05812F2296E3E00C94F259849B02C062
:1015400080E801C080E080934D050E94C41BFC012F
:1015500014821582168287B7806187BF81E08EBDB5
:101560000895A4E1B0E0E7EBFAE00C94C7590E94BB
:1015700071520E94B75668E070E080E090E00E94EF
:10158000FA52811102C0F12CF1C00E94FA516D870C
:101590007E878F87988B0E948856282E8F77082FFA
:1015A00010E020E030E009831A832B833C8399E02C
:1015B000892E912CA12CB12C312C412C512C320193
:1015C00028E030E040E050E02D833E834F83588791
:1015D000C12CD12C76012D853E854F8558898216E8
:1015E0009306A406B50608F0AFC00E948856B50160
:1015F000A401517066277727452B462B472B09F40A
:10160000A895482F4F7750E060E070E009811A817B
:101610002B813C81040F151F261F371F09831A8356
:101620002B833C83822587FD05C0C40ED51EE61E94
:10163000F71E84C014E7C11612E2D106E104F104DA
:1016400008F479C0A70196015695479537952795D7
:1016500029873A874B875C8729813A814B815C8156
:10166000241935094609570989859A85AB85BC85B2
:10167000281B390B4A0B5B0BA8EEB3E00E943F59C5
:1016800024E43CEA40E050E00E94EC5829013A0191
:10169000C701B6012EEF30E040E050E00E94EC5868
:1016A00075016401C21AD30AE40AF50AA70196017A
:1016B0008D819E81AF81B885281B390B4A0B5B0B4E
:1016C000298B3A8B4B8B5C8B33940E94A75660E03E
:1016D00070E0CB010E942753882309F454CF6D8119
:1016E0007E818F8198853DDB69897A898B899C8988
:1016F00038DBC301B20135DB0E9471520E94B7563C
:10170000C501B4016F5F7F4F8F4F9F4F0E94FA5208
:10171000882309F438CF49805A806B807C80098502
:101720001A852B853C85401A510A620A730ACD82BC
:10173000DE82EF82F886C12CD12C76011FEF811A50
:10174000910AA10AB10A47CF0E94A75660E070E053
:10175000CB010E942753F82E882309F414CF832D40
:101760000E946B520E9471520E94B7568F2D649650
:10177000E2E10C94E359CF93C82F97B79F7E97BFB0
:101780009EB59E7F9EBD1092840080E00E946B52A9
:1017900089E10E945A1F0E94651FC11103C0E1DE4A
:1017A000C82F01C0C1E00E94D7520E94C5528C2FA1
:1017B0008170CF91089581E0DECF0895849B03C0AE
:1017C00020E830E002C020E030E040914D0550E0DC
:1017D00081E02417350709F480E00895A0E1B0E026
:1017E000E4EFFBE00C94CA596C015B013A0149013A
:1017F000502E009719F480E090E065C061157105E6
:10180000D1F383E08017BCF307FF05C080912A0164
:101810008111F1CF1DC080E10802F0011124E254D2
:10182000FE4F9F2F990F990B80E1E82EF12C8E012E
:101830000F5F1F4F9F01492F592F692F792F892F34
:10184000F60109958823B9F28D818111DFCFD3CFBD
:1018500041E150E060E070E082E291E00E948C5A49
:10186000D0922301C0922201B0922501A0922401BE
:10187000709227016092260190922901809228019E
:1018800057FC1CC08D8180932A01CE0109960E94CD
:10189000085160932B0170932C0180932D0190933C
:1018A0002E01CE010D960E94085160932F01709376
:1018B0003001809331019093320103C08FEF809308
:1018C0002A0182E291E06096EFE00C94E6590097DD
:1018D00021F0FC01108681E0089580E008958435B0
:1018E00028F5603318F5262F269526952695E82F9E
:1018F000F0E0962F977034E5239FE00DF11D112441
:10190000E555FA4FA1E0B0E0092E01C0AA0F0A94F4
:10191000EAF7442319F090819A2B03C0A095908197
:101920009A239083262F482F0C94AD340895CF939B
:10193000DF93D82FC62F8435E0F46033D0F4262F00
:10194000482F0E94AD34EC2FE695E695E69584E5A8
:10195000E89FF0011124ED0FF11DE555FA4FC77016
:1019600081E090E001C0880FCA95EAF7908198273E
:101970009083DF91CF910895A3E0B0E0E2ECFCE02A
:101980000C94C859182F562E442EC82ED12C1B82C9
:101990001A824601840E911CA62EB12C3501620ECE
:1019A000711CEA81FB81EC0DFD1DE815F905DCF4E5
:1019B000E12CF12C3A80310EF701EA0DFB1DE61502
:1019C000F7055CF4652D6E0D402F832D298387DF8D
:1019D0008FEFE81AF80A2981EFCFEA81FB8131966F
:1019E000FB83EA83DECF2150250D4FEF440D410FDD
:1019F000652D812F0E94AD342396E1E10C94E459CA
:101A0000A0E0B0E0E6E0FDE00C94CC59182FB62E33
:101A1000842EA22EE82EF12CC0E0D0E06701C40E87
:101A2000D11C99249A94920E960EFE01EE0DFF1D84
:101A3000EC15FD0564F47C2E710E402F6B2D872D67
:101A40004EDF402F692D872D4ADF2196EECFEB2CFC
:101A5000F12CC0E0D0E06701CA0CD11C8A94782C2C
:101A6000710EFE01EE0DFF1DEC15FD0564F49C2EBC
:101A70009B0C402F692D812F32DF402F692D872D40
:101A80002EDF2196EECF2FEF2A0D2B0D482D410F83
:101A90006B2D812F0E94AD34CDB7DEB7EDE00C94F5
:101AA000E859A0E0B0E0E7E5FDE00C94D259D62E6D
:101AB000F82EC42FD0E0C80FD11D022F10E0060F62
:101AC000111D2F2D30E02C173D076CF4ED2C2E2D21
:101AD00030E0201731072CF46E2D8F2D28DFE39492
:101AE000F6CFF394EECFCDB7DEB7E7E00C94EE5926
:101AF0008FB9779BFECF779808958FEF8FB9779B3B
:101B0000FECF77988FB10895A4E0B0E0EAE8FDE059
:101B10000C94D659182F8FEF8FB9779BFECF7798FB
:101B20008FB1812F80644C835B836A837983E0DF8C
:101B30007981872FDDDF6A81862FDADF5B81852F50
:101B4000D7DF4C81842FD4DF112321F0183039F4F2
:101B500087E801C085E9CCDF9AE02FEF0AC08FEF5C
:101B6000FACF779BFECF77988FB18F3F21F49150BA
:101B700011F02FB9F6CF2496E3E00C94F259EF92CE
:101B8000FF920F931F938091350181111EC0209108
:101B900036013091370140913801509139016091FF
:101BA0003A0170913B01E12C82E0F82E0EE311E046
:101BB00080913C0190913D0180D2882321F081E009
:101BC0008093350103C080E001C081E01F910F9137
:101BD000FF90EF900895A8E1B0E0E1EFFDE00C94F4
:101BE000C75929833A834B835C836D837E838F83BC
:101BF00098874801FA8AE98A55245A9469897A892A
:101C0000672B09F41FC169807A8021E07222930159
:101C100040E050E060E070E0CB0169863A874B8796
:101C20005C876D877E878F87988B29813A814B816E
:101C30005C816D817E818F819885A984BA84C12C55
:101C4000D12CE12CF12C00E010E00E944A5A288FA0
:101C50003F8B4987452E6B8B7C8B8D8B9E8B212CEC
:101C600092E0392E2618370849895A8942155305BA
:101C700008F41A01A0903601B0903701C0903801E5
:101C8000D0903901E0903A01F0903B0100913C0185
:101C900010913D01288D3F894985542D6B897C89A0
:101CA0008D899E890E94535A29F48091330188239B
:101CB00009F49FC064DF882309F4C6C0A898809106
:101CC000340182FF0FC0288D3F894985542D6B89CF
:101CD0007C898D899E8909E00E94195ABA01422F98
:101CE000532F04C0488D5F896985742D81E10CDF15
:101CF000882341F0A89AA8C0779BFECF77988FB130
:101D00008E3F11F05FB8F8CF809133018823A1F1A5
:101D100061147104A9F4211452E0350689F4F40128
:101D200080E090E05FB8779BFECF77982FB121934A
:101D30000196811562E09607A9F77EEF971A48C0D1
:101D40009101260D371D80E090E05FB8779BFECFB4
:101D500077984FB18615970548F08217930730F4AE
:101D6000F4014083A4014F5F5F4F4A010196811542
:101D700052E0950751F72CC0EEE3F1E05FB8779B96
:101D8000FECF77988FB1819363E0EE33F607B1F71A
:101D9000788D709336018F89809337019985909360
:101DA000380140923901EB89E0933A01FC89F093C4
:101DB0003B012D8920933C013E8930933D01B301C5
:101DC000625C7E4FA101C4010E94835A820C931C65
:101DD0005FB8779BFECF77988FB15FB8779BFECFC8
:101DE00077988FB1A89A5FB8779BFECF77988FB11D
:101DF00009C0B301625C7E4FA101C4010E94835AF5
:101E0000820C931C49895A89421953095A8B498B70
:101E1000910140E050E060E070E080E090E0A98057
:101E2000BA80CB80DC80ED80FE800F8118850E9417
:101E3000355A29833A834B835C836D837E838F83FA
:101E40009887DCCE81E001C080E06896E2E10C94E6
:101E5000E359A0E0B0E0EFE2FFE00C94D159BA9A68
:101E6000B99AA09ABB98A89A83E58DB970981092F8
:101E70003401CAE042DEC150E9F7A898C0E0D2E0E0
:101E800040E050E0BA0180E03FDE813021F0219750
:101E90002097B1F751C04AEA51E060E070E088E075
:101EA00033DE182F147082FD11C027DE26DE25DEFA
:101EB00080FF8DC022DE8A3A09F089C0809134010A
:101EC000826080933401C0E0D0E825C040E050E05B
:101ED000BA0187E319DE40E050E0BA0189E214DE7E
:101EE00082FDF1CF809134018160EBCF81FD19C07B
:101EF000C12CD12C760140E050E0BA0187E304DE2A
:101F0000B701A60189E200DE182F117080FF16C00C
:101F10002197209789F080913401982F937031F7A1
:101F200006C0C12CD12CE12C30E4F32EE4CF40E0EC
:101F300050E0BA0181E0E7CFA89A48C0C0913401CF
:101F4000C1FF12C040E050E0BA018AE3DDDD882322
:101F500011F0A89A3CC0D1DD86FF03C0C460C093D5
:101F60003401CBDDCADDC9DD40E052E060E070E065
:101F700080E1CADDA89A81112AC08DB18C7F8DB90C
:101F8000709A8FEF809336018093370180933801E8
:101F90008093390180933A0180933B0180933C0107
:101FA00080933D0181E080933501E12C22E0F22E07
:101FB0000EE311E020E030E040E050E060E070E04F
:101FC00080E090E008DE11E0811101C010E0812F77
:101FD000CDB7DEB7E8E00C94ED59A2E1B0E0E3EF55
:101FE000FFE00C94C75919012A016B837C838D8310
:101FF0009E8318870F833701DA82C982BA86A98641
:102000000115110511F480E054C0E114F104D9F375
:1020100029813A812E153F05B0F349855A85452B14
:1020200091F3970140E050E060E070E0CB01EB8677
:102030003C874D875E876F87788B898B9A8B73017E
:102040000F8118859101A2016B817C818D819E8118
:10205000C2DD8823C1F27401810192014B815C8150
:102060006D817E818F819885E985FA850995882320
:10207000F9F09101A2016B817C818D819E81AB84FD
:10208000BC84C12CD12CE12CF12C00E010E00E948A
:10209000355A19012A016B837C838D839E832981A4
:1020A0003A81261937093A8329832615370538F6E8
:1020B00081E06296E2E10C94E359A0E1B0E0E3E64E
:1020C000F0E10C94C75929833A834B835C836D8379
:1020D0007E838F8398871E870D87FA86E986898598
:1020E0009A85892B09F494C089819A8191709C8783
:1020F0008B871C0129813A814B815C816D817E81B6
:102100008F8198855101C12CD12CE12CF12C00E05C
:1021100010E00E944A5A288B3F873A011B012C018C
:10212000812C52E0952EEB85FC858E1A9F0A8985BD
:102130009A858815990508F44C01A0903601B09055
:102140003701C0903801D0903901E0903A01F09009
:102150003B0100913C0110913D0128893F85A3017D
:10216000B101C2010E94535A69F109DD882309F4C3
:1021700059C0EB85FC85EF2BB9F48114F2E09F0682
:1021800099F42889209336018F85809337016092D6
:1021900038017092390120923A0130923B0140920D
:1021A0003C0150923D010EC0E12C42E0F42E0EE3C2
:1021B00011E028893F85A301B101C2010CDD811125
:1021C000E0CF30C0ED85FE85EE53F14089F4A8984C
:1021D0008091340182FF1EC028893F85A301B1018F
:1021E000C20109E00E94195ABA01422F532F15C0AB
:1021F000A4016D857E858B859C85825C9E4F0E94A7
:10220000835A1092350189859A8588159905F9F6C2
:1022100081E051C048895F85B30188E175DC88237E
:1022200019F0A89A80E047C08EEF62DC0EE311E05F
:10223000F80181918F015CDCF3E00E331F07C1F7D9
:102240008FEF56DC8FEF54DC2FEF2FB9779BFECF4B
:1022500077988FB18F3FC1F78FB9779BFECF779873
:102260008FB1A89A8D859E85880D991D9E878D8733
:10227000940140E050E060E070E080E090E0A980F0
:10228000BA80CB80DC80ED80FE800F8118850E94B3
:10229000355A29833A834B835C836D837E838F8396
:1022A0009887E985FA85E819F909FA87E987F1E05D
:1022B000F093350114CF6096E2E10C94E359ABE062
:1022C000B0E0E5E6F1E10C94C75929833A83742E16
:1022D000652E562E472E382E292E1D830C8347013E
:1022E000DF82CE82B986A8860115110511F480E03F
:1022F00061C02E813F81232BD1F331E03B83E11478
:10230000F10409F44AC01B8248C08114910409F405
:1023100049C0E884F98409811A81272D362D452D7D
:10232000542D632D722D8C819D81EE81FF81099545
:102330009B878A87892BB1F1FB81FF23A9F1EA846E
:10234000FB840C811D8129813A81472D562D652DF5
:10235000742D832D922DB1DE882349F2EA84FB840B
:10236000970140E050E060E070E080E090E0A980FC
:10237000BA80C72CD62CE52CF42C032D122D0E94EC
:10238000355A29833A83742E652E562E472E382EC1
:10239000292E8A859B85881A990A9B81992309F49D
:1023A000B4CFB7CF81E006C02A853B85821693065D
:1023B00030F69DCF2B96E2E10C94E359A0E0B0E01B
:1023C000E4EEF1E10C94CE59EC01009709F407C159
:1023D0004DE150E060E070E00E948C5AA89840E027
:1023E00050E0BA018AE090DB811155C086DB8E3F58
:1023F000E9F7DC2E0C2F1D2FB0E6EB2EF12C7DDB48
:10240000402F4D1950E04F30510598F5FA01EA5B25
:10241000FF4F0C942A5988832CC0F801808329C06F
:10242000F801818326C08A8724C090E0A0E0B0E054
:102430000E2C04C0880F991FAA1FBB1F0A94D2F745
:102440004B855C856D857E85482B592B6A2B7B2BB4
:102450004B875C876D877E870CC08295807F8F87D6
:1024600008C0282F22952F709F85922B9F878F70F1
:10247000888B0F5F1F4FF8E0EF1AF10880EDE81628
:102480008FEFF80609F0BBCF40E050E0BA0189E0D9
:102490003BDB882311F0A89AA2C02FDB8E3FE9F71F
:1024A000D12CB12CE12CF12CC12C912CAA24A39479
:1024B00024DBD11007C0B82EB294B694B694A3E032
:1024C000BA2286C09EE0D9120EC086FDA98E85FD77
:1024D000AA8E84FDAB8E8C7090E09595879595952E
:1024E00087958C8F75C0E1E0BE1226C0F7E0DF163D
:1024F00031F0DF1640F099E09D1510F404C08F73A1
:10250000FE2CEE24E82AE9E0DE1262C0FFEFEF1AAB
:10251000FF0A970140E050E060E070E080E090E06A
:1025200003E10E94FE59298B3A8B4B8B5C8B6D8BA0
:102530007E8B8F8B988F4CC0B1104AC097E0D91614
:10254000A9F19D1560F0E5E0DE1669F1F6E0DF1215
:102550003FC08370E82EF12CFE2CEE2439C099E0A8
:10256000D91699F1D91640F1EAE0DE1231C0881F80
:102570008827881FC82A870120E030E0892D90E055
:102580008C0D911D029604C0000F111F221F331FD6
:102590008A95D2F7098B1A8B2B8B3C8B1D8A1E8A4E
:1025A0001F8A188E15C08F70982E12C0E82AEE0C64
:1025B000FF1CEE0CFF1C0CC08295869586958370DF
:1025C000E82AFFEFEF1AFF0A03C08370C82ECC0C75
:1025D000D39482E1D8126CCFA89A81E001C080E048
:1025E000CDB7DEB7EBE00C94EA59809151058370CA
:1025F0000895E1E5F5E0837090819C7F982B9083AE
:102600000895809151058695869583700895E1E53A
:10261000F5E08370880F880F9081937F982B9083CB
:1026200008958091510586FB882780F90895E1E59A
:10263000F5E0908180FB96F9908308958091510593
:1026400087FB882780F90895E1E5F5E0908180FB1C
:1026500097F9908308958091520581700895E2E57D
:10266000F5E0908180FB90F9908308958091510569
:102670008295837008958370282F2295207F9091F2
:1026800051059F7C922B90935105813011F4D8987D
:102690000895811101C0D89A0895809161059091A3
:1026A0006205089590936205809361050895809175
:1026B0005E0590915F05089590935F0580935E0598
:1026C0000895809158059091590508959093590562
:1026D00080935805089580915A0590915B0508955F
:1026E00090935B0580935A05089580914E059091D3
:1026F0004F05089590934F0580934E05089580915E
:102700005605909157050895909357058093560567
:10271000089580915205869581700895E2E5F5E06F
:10272000908180FB91F99083089580915305909159
:10273000540508959093540580935305089580930C
:1027400050050C94F33508958091500508958CEA56
:102750009DE090935F0580935E0584EA96E09093F8
:102760006205809361058BE692E090935905809312
:1027700058058EEB90E090935B0580935A0589ECA9
:1027800090E090934F0580934E0584EF90E09093F6
:10279000570580935605E2E5F5E080818D7F8083C3
:1027A0008FED97E0909354058093530510925D054B
:1027B00010925C0580E580935005089542E050E05A
:1027C00060E070E081E595E00E946C5D90915105BC
:1027D000892F837092959370933019F090E002974F
:1027E0006CF0B5DF80915105837F8093510582E0C5
:1027F00042DF809151058C7F809351058091510576
:102800008295837038DF84E090E00E94845D9C01B3
:10281000245F31402D31354218F4282F892F02C012
:102820002CEA8DE020935E0580935F0586E090E0C2
:102830000E94845D9C01245F31402539314118F4A8
:10284000282F892F02C024EA86E020936105809317
:10285000620588E090E00E94845D9C01225331096A
:102860002F39374018F4282F892F02C02BE682E039
:1028700020935805809359058AE090E00E94845D7A
:102880009C0122533109273B334018F4282F892F0C
:1028900002C02EEB80E020935A0580935B058CE00C
:1028A00090E00E94845D9C0122533109273B334014
:1028B00018F4282F892F02C029EC80E020934E05C0
:1028C00080934F058EE090E00E94845D9C0122532E
:1028D0003109273B334018F4282F892F02C024EFF9
:1028E00080E0209356058093570580E190E00E9498
:1028F000845D9C01205D37402536310518F4282F72
:10290000892F02C02FED87E0209353058093540553
:1029100082E190E00E94845D803D2AE8920724F0E5
:10292000813345E794071CF020E080E002C0282FA7
:10293000892F20935C0580935D0583E190E00E94E0
:102940007C5D813808F080E580935005089542E071
:1029500050E060E070E081E595E00E94895D609163
:102960005E0570915F0584E090E00E94A95D609132
:1029700061057091620586E090E00E94A95D60911A
:1029800058057091590588E090E00E94A95D60911A
:102990005A0570915B058AE090E00E94A95D609104
:1029A0004E0570914F058CE090E00E94A95D60910A
:1029B0005605709157058EE090E00E94A95D6091E8
:1029C0005C0570915D0582E190E00E94A95D6091D7
:1029D000500583E190E00C94985D089580E090E0CC
:1029E0002091740027FD03C001970097C9F708954F
:1029F0001092710088E480937000089584EA8093B7
:102A00007400ECDF90917100987F81E0983009F0BC
:102A100080E00895CF9380FD02C0C8E101C0C0E40A
:102A20008093730084E880937400D8DF4091710034
:102A3000487F50E02C2F30E081E04217530709F027
:102A400080E0CF9108958093730084E880937400B0
:102A5000C5DF90917100987F81E0983209F080E0A5
:102A60000895CF93DF93EC0184EC80937400B6DF7C
:102A700090917100809173008883987F81E09035F8
:102A800009F080E0DF91CF910895CF93DF93EC01BF
:102A900084E880937400A2DF9091710080917300AC
:102AA0008883987F81E0983509F080E0DF91CF91AD
:102AB000089584E98093740080E090E02091740090
:102AC00024FF05C001970097C9F780E0089581E0D1
:102AD00008956AE070E088EE93E00C94D34F089577
:102AE000CF939A9908C0809165058F3F31F08F5F31
:102AF0008093650502C0109265059E9908C080917B
:102B000066058F3F31F08F5F8093660502C010929B
:102B100066059B9908C0809163058F3F31F08F5FF8
:102B20008093630502C0109263059D9908C080914F
:102B300064058F3F31F08F5F8093640502C010926F
:102B400064059C9908C0809167058F3F31F08F5FC5
:102B50008093670502C01092670563DDC82F8091DE
:102B60006505853039F482E00E94DD2BCC2311F01D
:102B7000B0DFC0E080916605853039F483E00E94C3
:102B8000DD2BCC2311F0A5DFC0E0809163058530FB
:102B900039F480E00E94DD2BCC2311F09ADFC0E0F5
:102BA00080916405853039F481E00E94DD2BCC23CF
:102BB00011F08FDFC0E080916705853029F484E053
:102BC0000E94DD2BC11185DFCF91089584B38C67FE
:102BD00084BB85B38C6785BB109265051092660532
:102BE0001092630510926405109267050895E82F0E
:102BF000F0E0ED59FA4F81E09081933308F480E0E2
:102C00000895A0E1B0E0E7E0F6E10C94C759782E12
:102C1000698380916C05481720F090916D05941799
:102C200008F44EE290916E0591114EC0672CE42E8F
:102C3000F12CC72CD12C2981A22EB12C962D9719BD
:102C400080916A05981708F07FC120916C05B70143
:102C5000621B7109869FA001879F500D1124490FA7
:102C6000511DE0916805F0916905E40FF51F04918D
:102C7000812C912C2601490E511C10E034E543169D
:102C800051040CF05EC194012A0D3B1D2033310527
:102C90000CF057C16981680D9801082C02C0359568
:102CA00027950A94E2F720FF02C041E001C040E00E
:102CB000862D0E946F0C8FEF881A980A98E089166B
:102CC0009104E1F66394BACF913009F092C040903C
:102CD0006B054694469446944394E42EF12CE81AEE
:102CE000F10820916A05429E202D11242F5F2E9D10
:102CF000C0012F9D900D1124E0916805F0916905A8
:102D0000E80FF91F24912A83242D30E03D832C8382
:102D10004F01E12CF12C272D30E03B872A873981A8
:102D2000232F30E03D872C876E2C3A81E31608F084
:102D30000AC100E010E0C12CD12C94012F5F3F4F5D
:102D40003F832E832A853B852E0D3F1D398728879B
:102D5000670CEE81FF81EC0DFD1DA4905980500E93
:102D6000188A1F862C843D84200E311EB12C2885A4
:102D70003985243531050CF0E4C08F852F853889DD
:102D8000220D331D203331050CF0DBC020916B0583
:102D900030E04F855889400F511F4217530784F484
:102DA000D50102C0B595A7958A95E2F76F85650DA7
:102DB000A0FF02C041E001C040E0862D0E946F0CE0
:102DC0002F8538892F5F3F4F388B2F87283031056B
:102DD00071F63FEFC31AD30A085F1F4FC41408F4FB
:102DE000B8CF8FEFE81AF80A2C813D81820E931E2E
:102DF0009BCF923009F0A5C090916B059695969562
:102E000096959F5F60916A05E42EF12CE81AF1080F
:102E1000969F802D11248E9D90018F9D300D112441
:102E2000E0906805F0906905E20EF31EAFEFA60F83
:102E300080E0462F50E041505109262E281AB42F29
:102E4000B81B70E030E0F701E70FF11DE0813F5F54
:102E50007B0F3917C0F3E11105C08A1711F08F5F9E
:102E6000ECCF212C00E010E0C12CD12C272D30E03C
:102E70003D832C833981232F30E03F832E8369806B
:102E8000600E412C512C2E813F81200F311F3B833E
:102E90002A83342C421408F04AC080916A058C9D24
:102EA000F0018D9DF00D1124E40DF51DEE0DFF1DBB
:102EB000849019861886AC80BD80A40CB51C912C1A
:102EC000370C84E5A816B104E4F548856A817B8156
:102ED00028853985620F731F6033710594F5609101
:102EE0006B0570E0F901E00FF11FE617F70794F4A6
:102EF000D40102C0B595A7954A95E2F7622F660DF9
:102F0000A0FF02C041E001C040E0832D9E870E94E7
:102F10006F0C9E85288539852F5F3F4F398728871D
:102F20002830310571F63FEF431A530AB2CF8FEFC5
:102F3000C81AD80A085F1F4FC91608F4A0CF822DFF
:102F400003C080E001C08A816096E2E10C94E359FD
:102F50000F931F93CF93DF93182F062FE62FF0E0E8
:102F600080916B052FE230E0281B31092E173F07B7
:102F700054F0EA014991442331F0602F812F41DE62
:102F80008F5F180FF7CF812FDF91CF911F910F9196
:102F900008950F931F93CF93DF93182F062FE62FDB
:102FA000F0E080916B052FE230E0281B31092E17ED
:102FB0003F076CF0FA014491EF012196442339F068
:102FC000602F812F1EDE8F5F180FFE01F4CF812F3F
:102FD000DF91CF911F910F91089587B78F7E87BFA3
:102FE0000E94F5500E94C552109284001B98809157
:102FF0003005882321F061E083E05FD703C081E0E2
:103000008093400362C70895CF92DF92EF92FF92C0
:10301000CF93DF9300D000D0CDB7DEB70E940F541E
:10302000882309F488C00E949A560E949906623546
:1030300079448644964409F07BC00E9499060E9418
:103040009906673571448645954409F071C00E9420
:10305000990666367D468447904209F069C00E9411
:103060009906603171058105910509F061C00E94E2
:103070008F06019709F05CC00E948F06019709F046
:1030800057C00E9499069B01AC0169833A834B8328
:103090005C830E94990629813A814B815C812617C5
:1030A00037074807590709F043C00E948F060E945E
:1030B0008F060897E9F50E949906643671468447A1
:1030C0009146B1F50E9499066B017C011FBC60E03E
:1030D00074E284EF90E029813A814B815C810E9407
:1030E000EC583093740520937305C0926F05D0920D
:1030F0007005E0927105F09272051DBC1CBC8091B8
:103100007305909174059BBD8ABD89EE97E09093FD
:103110007705809376058DEE97E19093C8078093AD
:10312000C70787B7806187BF81E08EBD80E004C09C
:1031300054DF82E001C081E00F900F900F900F905C
:10314000DF91CF91FF90EF90DF90CF9008951F9285
:103150000F920FB60F9211240BB60F922F933F933D
:103160004F935F936F937F938F939F93AF93BF938F
:10317000EF93FF930E94A73BFF91EF91BF91AF9117
:103180009F918F917F916F915F914F913F912F917F
:103190000F900BBE0F900FBE0F901F9018951F92AF
:1031A0000F920FB60F9211240BB60F922F933F93ED
:1031B0004F935F936F937F938F939F93AF93BF933F
:1031C000EF93FF930E942008FF91EF91BF91AF9181
:1031D0009F918F917F916F915F914F913F912F912F
:1031E0000F900BBE0F900FBE0F901F9018951F925F
:1031F0000F920FB60F9211240BB60F922F933F939D
:103200004F935F936F937F938F939F93AF93BF93EE
:10321000EF93FF930E94EC08FF91EF91BF91AF9164
:103220009F918F917F916F915F914F913F912F91DE
:103230000F900BBE0F900FBE0F901F9018951F920E
:103240000F920FB60F9211240BB60F922F933F934C
:103250004F935F936F937F938F939F93AF93BF939E
:10326000EF93FF9383B5845683BD8091750581608C
:10327000809375059CD2FF91EF91BF91AF919F9183
:103280008F917F916F915F914F913F912F910F900F
:103290000BBE0F900FBE0F901F9018951F920F92AC
:1032A0000FB60F9211248F939F9384B195B1909391
:1032B0007905809378059F918F910F900FBE0F90A5
:1032C0001F90189585B7837E85BFA09A8F98139A13
:1032D000149A119A8C98D09A949A979A87E487B9FD
:1032E0008EEC86B98FEF9FEF9093790580937805E8
:1032F0000E94F5500E948B562FE088E190E00FB6B7
:10330000F894A89581BD0FBE21BD66E970E088EEF6
:1033100093E00E94D34F34D2A89550DAA895B3D049
:1033200086E40E94F33510DA0E94F3350E94D93406
:1033300064E670E080ED97E00E94D34FA89585B5D4
:10334000856085BD87B7806887BF85E191E00E9471
:103350008D5160E070E0CB010E948354A895789471
:1033600035DC9C993BC09A9939C09E9937C062E37D
:1033700070E088EE93E00E94D34F6EE170E08CED38
:1033800095E00E94D34F64E170E080ED97E00E94E9
:10339000D34F6EE170E08CED95E00E94D34F62E375
:1033A00070E088EE93E00E94D34F62E370E08CEB14
:1033B00092E00E94D34F9C9909C0A89568EE73E0F3
:1033C00088EE93E00E94D34FA895F5CF9A9BF5CF56
:1033D0009E9BF3CF1092A60582E16CD510927505E5
:1033E00074D5A89543D9813009F0D89AC8EED3E0B6
:1033F00037E4F32E4EECE42E0FEF1FEF80917505AE
:1034000080FF3AC0809175058E7F80937505A895E1
:1034100067DB2CD9823071F483B38C778C3721F041
:10342000D898C4EFD1E006C0209721F021972097CB
:1034300009F4D89A8091780590917905019681F0E8
:1034400080917805909179059695879596958795C1
:1034500080930701F7B8E6B81093790500937805D3
:1034600080913E03863020F48F5F80933E0304C03A
:1034700010923E030E9442340E945D530E94C6395E
:103480000E940E0ABBCFB89ABA9ABD9AB99ABD9A51
:10349000BC9ABE9AC59A80E58DB91EB80E944F3677
:1034A00067EA75E08BEA95E00E94FA340C94D9340F
:1034B0000895C5988FB98FEF779902C08150E1F7D1
:1034C000C59A0895C598C69880EA9FE00197F1F7DC
:1034D000C69AC59A0895CF93DF93EC0189DA8EDA04
:1034E000811103C0E6DA80E051C080EA93DA8823D4
:1034F000C9F381E0A8DA8823A9F3DBDA882391F302
:103500007DDA882379F381EA85DA882359F3CE01BD
:103510000696A7DA882331F3CE010596A2DA88232E
:1035200009F3CE0104969DDA8823E1F2CE010396D9
:10353000ACDA8823B9F2BDDA8823A1F29E81292F63
:1035400022952F709F703AE0239F900D11249E8347
:103550009D81292F22952F709F703AE0239F900D17
:1035600011249D839C81292F22952F709F703AE012
:10357000239F900D11249C839B81292F22952F70CE
:103580009F703AE0239F900D11249B83DF91CF9190
:1035900008951F93CF93DF93EC012ADA2FDA81117C
:1035A00003C087DA80E03EC080EA34DA8823C9F3BA
:1035B00081E049DA8823A9F38E811AE0612F0E9405
:1035C000B95820E1829F900D1124892F3CDA88237D
:1035D00041F38D81612F0E94B95820E1829F900DA7
:1035E0001124892F30DA8823E1F28C81612F0E9427
:1035F000B95820E1829F900D1124892F24DA882365
:1036000081F28B81612F0E94B95820E1829F900D39
:103610001124892F18DA882309F4C3CF4ADA8823C2
:1036200009F4BFCFDF91CF911F910895A2E0B0E0E0
:10363000ECE1FBE10C94D5598C01DAD9DFD9811189
:1036400003C037DA80E03FC080EAE4D98823C9F3B9
:1036500085E0F9D98823A9F32CDA882391F3CED910
:10366000882379F381EAD6D9882359F3CE010296CB
:10367000F8D9882331F3CE01019607DA882309F3BC
:1036800018DA8823F1F23A81932F929596959695C0
:103690009370F8019083498144FB222720F9220F7F
:1036A000922F990F990F920F4F70940F9183232FA0
:1036B0002695269526952670922F990F990F920F91
:1036C0003F70930F92832296E4E00C94F1590F938C
:1036D0001F93CF93DF93EC018BD90A811881D98195
:1036E0008DD9811103C0E5D980E029C080EA92D943
:1036F0008823C9F385E0A7D98823A9F3CAE0802FDE
:103700006C2F0E94B95820E1829F900D1124892FBF
:1037100090E4199F90011124822B95D9882319F3E5
:103720008D2F6C2F0E94B95820E1829F900D11249B
:10373000892F89D98823B9F2BCD98823A1F2DF91D6
:10374000CF911F910F910895CF93DF93EC016EDF1E
:10375000882319F0CE01BFDE01C080E08170DF91C7
:10376000CF910895CF93DF93EC01B1DF882319F057
:10377000CE010FDF01C080E08170DF91CF9108950D
:103780008AE795E0E1CF08958AE795E00895DC01A6
:103790001196EC911197E23019F48C91837029F015
:1037A000F0E0EA58FE4F849108958DE10895CF939B
:1037B000809180058F5F809380058436C0F11092E0
:1037C000800580917F058F5F80937F058C3378F132
:1037D00010927F0580917E058F5F80937E058C33EC
:1037E00030F110927E0580917D058F5F80937D057D
:1037F0008831E8F010927D05C0917C05CF5FC093C1
:103800007C058AE795E0C3DF8C1788F491E09093FC
:103810007C0580917B058F5F80937B058D3038F030
:1038200090937B0580917A058F5F80937A05CF9185
:103830000895A7E0B0E0EFE1FCE10C94CB596C01F6
:103840004B015A013901CE0101967EDF0E9495138A
:103850002981820F911DF601918380838A81F40171
:1038600080838B81F50180838C81F30180838D813E
:10387000F80180838E81F70180832796EEE00C9417
:10388000E7591092800510927F0510927E051092E4
:103890007D050895AC0167E280E07BCB0895A0E050
:1038A000B0E0E5E5FCE10C94CD59982E862E7A0126
:1038B00005E010E0B12C40E0C0E1D7E28AE0C82E7C
:1038C000D12CC701BE010E94C558A62E611105C0AA
:1038D000411103C0C130D10549F440E34A0D682DC0
:1038E0008B2D890D8ED9B394B80E41E0AC9E90011A
:1038F000AD9E300D1124E21AF30ACE01B6010E94EA
:10390000C558EB010150110901151105D1F68B2D98
:10391000CDB7DEB7ECE00C94E959A1E0B0E0E3E903
:10392000FCE10C94D459082FF62E842F6AE00E94F3
:10393000B95840E3480F6F2D802F998362D911E069
:10394000180F998140E3490F6F2D812F800F59D9AE
:103950008F5F810F2196E5E00C94F0594F925F92B2
:103960006F927F928F929F92AF92BF92EF920F933E
:10397000CF93DF934B015C0129013A01D02F60EF17
:1039800070E080E090E0A50194010E94EC58C22F05
:10399000233008F4C3E0A0E3B0E0A30192010E9449
:1039A0003F59A50194010E94EC58622FEC2FF0E0E2
:1039B000E20FF11DF19714F060E36C1B01E02C2F76
:1039C0004E2D8D2F0E94BC0CDF91CF910F91EF9067
:1039D000BF90AF909F908F907F906F905F904F902F
:1039E00008958091A605833091F038F4882361F022
:1039F000813099F4C9DE01960895843059F08530FC
:103A000061F4C2DE05960895BFDE02960895BCDE1D
:103A100003960895B9DE0496089580E090E0089535
:103A2000CF93DF93EC010E947A5A982F990F980F49
:103A3000990FAE0167E284E5891BABDADF91CF9184
:103A400008951F93CF93DF93EA01E82FF0E02091D0
:103A5000820530918305E217F307E0F0C90105966E
:103A6000E817F907B8F4E21BF30B19E0E19F102DFA
:103A700011241F5FAB01612F83E08BDACE010E941E
:103A80007A5A982F990F980F990FAE01612F84E5FC
:103A9000891B7FDADF91CF911F910895FF920F93D9
:103AA0001F93CF93DF93D82FC92FF62E042F0E9498
:103AB0007A5A482F5BEF5403900111242C5A3F4F40
:103AC000E1E0F0E0E81BF1090E9FD0010F9FB00D7F
:103AD00011242A0F3B1F37FF02C02F5F3F4F359540
:103AE0002795122FED2FFC2F4491EF0121964423AF
:103AF00039F06F2D812F85D8800F180FFE01F4CF7C
:103B0000CDB7DEB7E5E00C94F0590F931F93CF9338
:103B1000DF932091A6058091820590918305820F05
:103B2000911D892B19F40E94875125C0C0E0D0E077
:103B300000E010E00E9487518C0F9D1FFC018081E6
:103B40002196811112C00F5F1F4F8091A605209111
:103B5000820530918305280F311D0217130729F4C0
:103B60000E9487518C0F9D1F06C0C632F2E0DF070E
:103B700009F780E090E0DF91CF911F910F910895B8
:103B800090918E05992391F0482F50E09091A605D1
:103B90002091820530918305290F311D421753076B
:103BA00029F480918F05909190050895823099F0C5
:103BB00038F4882369F08130B9F40C944D130895DA
:103BC000843079F058F0853079F40C947F1308959F
:103BD0000C94571308950C94611308950C946B136F
:103BE00008950C947513089580E090E00895A1E085
:103BF000B0E0EDEFFDE10C94C959182F7A01482E81
:103C0000512C20918205309183054216530608F409
:103C100072C0A9014B5F5F4F4416550608F06BC098
:103C2000C201821B930B9C0189E0289F902C1124D8
:103C30009394AB01692D83E0ACD9812FA1DF482F8C
:103C4000892EC70149830E947A5A6C014981E42F69
:103C5000F82D05E010E0712C612C20E137E25AE0EC
:103C6000A52EB12CCF01B9010E94C558611105C024
:103C7000611003C02130310519F4739466246394F4
:103C8000629FD001639FB00D1124EA1BFB0BC90199
:103C9000B5010E94C5589B0101501109011511057C
:103CA00009F79601270D311D122F110F120F110F59
:103CB000582D692D82E5811BF2DD8C5AA701692DF3
:103CC000811B67D980918E058823A9F02091A605D4
:103CD0008091820590918305820F911D48165906A7
:103CE00051F469E0269F602D11246F5F4DE951E08A
:103CF0008CE4811B4ED92196E0E10C94E5590E9499
:103D0000CC510E94985360E070E0CB010E94835434
:103D100010928305109282051092A6050895CF9205
:103D2000DF92EF92FF921F93CF93DF93CDB7DEB771
:103D3000A0970FB6F894DEBF0FBECDBF0E94995179
:103D400030E040E051E0530FFC01E30FF11D308102
:103D50003323C1F03F3229F4198220E0352F422F5E
:103D6000F1CF21E0240FE1E0F0E0EC0FFD1FE40FC4
:103D7000F11D3083E1E0F0E0EC0FFD1FE20FF11DDB
:103D80001082ECCF0E94B451182F882309F44BC045
:103D90000E94CC510E949853CE0101960E949E55DC
:103DA0006B017C0110928305109282051092A6058A
:103DB0008FEFC816D806E806F80671F10E948A51FE
:103DC000FC0142815381648175814550510961092B
:103DD00071094C155D056E057F0508F50E948A5135
:103DE000FC0182819381A481B5810697A105B1056B
:103DF00088F00E948A51FC0142815381648175815F
:103E00004550510961097109C41AC092A6056A0199
:103E10007B0105C0C092A605C12CD12C7601C7013B
:103E2000B6010E948354812FA0960FB6F894DEBF8E
:103E30000FBECDBFDF91CF911F91FF90EF90DF902C
:103E4000CF900895FF920F931F93CF93DF93EC01D0
:103E5000062F0E94CD5A8031A8F4482F5BEF5403FF
:103E6000900111242C5A3F4F41E050E0481B51096A
:103E7000240F351F37FF02C02F5F3F4F3595279521
:103E8000122F01C010E080E0FF24F394F80EFE0131
:103E9000E80FF11D4081442341F0602F812F0E94E3
:103EA00001168F5F180F8F2DEFCFCDB7DEB7E5E08E
:103EB0000C94F05980934003089580938C0560938F
:103EC000810583E1809340030895ACE1B0E0EBE627
:103ED000FFE10C94C75980914003843129F407B65F
:103EE00004FE02C00C94D92B0FEF20E247E065E0FE
:103EF00087E498E00E94DA350E94EA34809140031A
:103F000090E08A31910510F00C94D72BFC01EB5A0C
:103F1000FF4F0C942A590E940E0A60E085E995E053
:103F200091DF0E942C0AFC0100810E94F512811190
:103F300003C042EF57E002C04DEE57E069E080E079
:103F400028D8182F85E0810FBAE0EB2EE10E013062
:103F500049F541E050E069E0A2DC1E2D180F0E94F7
:103F60002F0A813051F40E94F512811103C047E2FB
:103F700055E016C041E255E013C00E942C0AFC0136
:103F80004181528169E0812F8ADC1E5F180F0E94F7
:103F9000F512811103C04FE155E002C04DE155E03B
:103FA00069E059C010E0A8014150510969E077DC8F
:103FB000E80E0E942C0AFC014381548169E08E2D99
:103FC0006EDCA2E0FA2EF80EFE0C0E94F5128111B2
:103FD00003C04FE155E002C04DE155E069E08F2D8F
:103FE0000E94C9170E94F512811103C042EF57E0E9
:103FF00002C04DEE57E062E180E00E94C917F5E093
:10400000FF2EF80EA80162E18F2D49DC15E0180F94
:104010001F0D0E942F0A813051F40E94F512811168
:1040200003C047E255E016C041E255E013C00E94CC
:104030002C0AFC014181528162E1812F30DC1E5F3C
:10404000180F0E94F512811103C04FE155E002C024
:104050004DE155E062E1812F0E94C9170E94F512DF
:10406000811103C082E498E002C08DE398E012DC85
:104070000E940E0A0C94D72B60E085E995E0E2DE01
:1040800001E027E044E56AE080E00E94000D0E9424
:10409000973B9B01AC01A0E5B0E00E943F59209105
:1040A00088053091890540918A0550918B050E94C1
:1040B000EC58422F23E06CE082E00E94BC0C80911F
:1040C000BB07882309F444C00E94F512811103C084
:1040D00042EF57E002C04DEE57E063E180E00E94FE
:1040E000C917182F0E94A03B81110AC04091BB073D
:1040F00050E063E185E0810FD2DB195F180F1CC02F
:1041000043DBFC018681893138F09DEC980F81E01A
:10411000983118F080E001C081E080FDE7CF809108
:10412000BB078A3010F4135F07C08091BB07843649
:1041300010F41D5E01C0175E4FE263E1812F0E9403
:104140000116810F4091BC0750E063E18E5FA7DB51
:104150000E94A03B882369F00E94F512811103C0E0
:1041600087E398E002C081E398E041E06DE196DCEE
:1041700031C00E94973B00918805109189052091DC
:104180008A0530918B05601771078207930768F4E1
:10419000FBDAFC011481F8DAFC010581F5DAFC0197
:1041A0001083F2DAFC01018306C0EEDAFC01108113
:1041B000EBDAFC010181412F6DE18DE1AEDB1DE108
:1041C000180F4AE36DE1812F0E940116402F6DE127
:1041D000810FA3DB0E94973B009188051091890510
:1041E00020918A0530918B0560177107820793072C
:1041F00010F00C94832B0E94F512811103C082E40D
:1042000098E002C08DE398E045DB0E94A03B0C944F
:104210006B2B0E94F512811103C083E897E002C066
:1042200089E797E041E061E039DC0E94F5128111F5
:1042300003C084E797E002C08AE697E041E06AE0C5
:104240002DDC0E94F512811103C081E697E002C0C7
:1042500087E597E041E063E121DC0E94F5128111DE
:1042600003C08FE497E002C086E497E041E06CE190
:1042700015DC0E94F512811103C080E497E002C0B2
:104280008BE397E041E065E209DC0E94F512909132
:10429000A60569E0969F602D112429E0811103C0D5
:1042A00046E38FE002C040E48AE00E94510D0E9484
:1042B0009256882311F40C94D72B0E949256482FC3
:1042C00050E060E080E0EBDA0E949556AC016AE0D5
:1042D00080E00BC141E060E089E595E0DFDB41E093
:1042E00069E082E595E0DADB40E062E182E495E0B6
:1042F000D5DB41E06BE18DE395E0D0DB40E064E2AB
:104300008DE295E00C94D52B0E948A51FC018281AC
:104310009381A481B581892B8A2B8B2B69F40E9410
:10432000F512811103C083EB97E002C08BEA97E09E
:1043300041E060E00C94D52BDD24D394CC24C394CD
:10434000E12CF12C712C00E010E00E948751800FCD
:10435000911FFC014081FBE0F71578F40E94875122
:10436000800F911FFC018081882319F00F5F1F4F80
:10437000F5CF01501109712C77C0411167C0FFEFD3
:10438000EF1AFF0A0E948A51A70160E070E0FC0169
:1043900082809380A480B580481559056A057B0505
:1043A00008F441C06091A60589E0689F602D112442
:1043B00029E04DE480E00E94510D0E948A51FC01E9
:1043C00082819381A481B5810697A105B10510F47E
:1043D0000C94D72B00E020E343E060E081E50E94ED
:1043E000BC0C0E948A516091820570918305FC018A
:1043F0002681378140855185260F371F411D511D6C
:104400002C8F398F4A8F5B8F0E948A51FC01628109
:10441000738184819581E2E0EE2E02E52C8D398D49
:104420004A8D5B8D57C22091820530918305C90169
:104430000596E816F90608F0B5CF2E153F05A0F44D
:10444000F9E0CF0E712CDD24D3940EC0809182054B
:1044500090918305E816F90638F06C2D8D2D0E9499
:104460000116D394D80E73940F5F1F4F063222E0CB
:10447000120708F46ACF96CF45E955E060E080E086
:104480000E94A8170E94F512811103C040EE57E068
:1044900002C040ED57E069E080E00E94C9178091BA
:1044A0009205833011F00C94D72B0E94F5128111E4
:1044B00003C042EF57E002C04DEE57E064E180E0F8
:1044C0000E94C9174091910550E064E183E2E7D969
:1044D00015E2180F4FE264E1812F0E94011640910E
:1044E000BC0750E08E5F64E1810FD9D90C94D72BC3
:1044F0000E94F512811103C083E895E002C08AE7AB
:1045000095E041E069E0CADA0E94F512811103C02A
:104510008DE695E002C082E695E041E062E1BEDA18
:104520000E94F512811104C088E198E00C94BA2B26
:1045300081E198E00C94BA2B60E085E995E082DC9B
:104540000E94F512811103C04AE055E002C043E029
:1045500055E069E080E00E94C917182F0E942C0ADC
:10456000FC01408150E069E085E0810F98D980909E
:10457000880590908905A0908A05B0908B0508E089
:1045800010E0312C212C50E8C52E56E9D52E58E9E3
:10459000E52EF12C6AE0462E512C612C712CC501C0
:1045A000B401A70196010E94EC58211108C0211006
:1045B00006C0F1E0CF16D104E104F10461F440E358
:1045C000420F62E1832D2C8F0E9401163394380E26
:1045D000222423942C8DA22FB0E0A70196010E94E3
:1045E0003F59861A970AA80AB90AC701B601A3015A
:1045F00092010E94EC5869017A01015011090115DC
:10460000110569F615E0130D0E94F512811103C022
:1046100047E155E002C042E155E062E1812F0E948E
:10462000C91780919205823071F40E94F5128111B0
:1046300003C040EE57E002C040ED57E06BE180E080
:104640000E94C9171BC08330C9F40E94F512811162
:1046500003C046EC57E002C04BEB57E06BE180E053
:104660000E94C917182F4AE36BE10E940116810FBF
:104670004091910550E06BE18B5F11D90E94F512DA
:10468000811104C08EEF97E00C94BA2B88EF97E06D
:104690000C94BA2B0E94F512811107C00E94F512EA
:1046A00081110AC006E616E00CC00E94F5128111C5
:1046B00006C00EE516E005C002E616E002C00AE5F7
:1046C00016E00E94F512811103C062E377E002C098
:1046D0006DE277E0A80180E0B4D90E94111388232D
:1046E00039F00E94F51281110AC00CE816E00CC0E6
:1046F0000E94F512811106C004E816E005C008E822
:1047000016E002C000E816E00E94F512811103C015
:1047100063E277E002C068E177E0A80181E091D927
:104720000E941E13882339F00E94F51281110AC0DD
:104730000CE816E00CC00E94F512811106C004E8D6
:1047400016E005C008E816E002C000E816E00E9486
:10475000F512811103C06DE077E002C062E077E0FE
:10476000A80182E06ED90E942B13882339F00E94A1
:10477000F51281110AC00CE816E00CC00E94F51277
:10478000811106C004E816E005C008E816E002C082
:1047900000E816E00E94F512811103C068EF76E090
:1047A00002C06EEE76E0A80183E04BD90E9436137A
:1047B000882349F0813071F40E94F512811111C0F3
:1047C0000CE816E016C00E94F51281110DC004E835
:1047D00016E00FC00E94F512811109C00BE716E028
:1047E00008C008E816E005C000E816E002C006E7C9
:1047F00016E00E94F512811103C064EE76E002C05B
:104800006AED76E0A80184E01CD90E940113815072
:10481000833048F4E82FF0E0EE0FFF1FE95EFE4F13
:104820000081118102C003E716E00E94F512811198
:1048300003C064ED76E002C06BEC76E0A80185E091
:1048400000D90E94F512811103C063EC76E002C02A
:104850006AEB76E04BE951E086E0F3D80E94F5126E
:10486000811103C06EEA76E002C061EA76E04BE9AE
:1048700051E087E0E6D80E94F512811103C068E993
:1048800076E002C06FE876E04BE951E088E0D9D8E5
:104890006091A60589E0689F602D112429E042E51A
:1048A00082E00E94510D00E020E342E060E080E001
:1048B0000E94BC0C8091A605209182053091830551
:1048C000280F311D40E050E0EE24E3946DE070E0ED
:1048D00080E090E043D86BC78091A605813009F451
:1048E000A1C038F0823009F4F6C0833009F463C106
:1048F00007C20E94F512811103C08AEF94E002C042
:104900008DEE94E041E060E0C9D80E94F51281117B
:1049100003C08AEF94E002C08DEE94E09F938F93E2
:104920008E010F5F1F4F1F930F930E94505B0E94D9
:1049300062562AE0A8010E94085B6DE174E0C8019C
:104940000E94685A0E9475562AE0AE014F5E5F4F82
:104950000E94085BBE016F5E7F4FC8010E94935AA0
:1049600069E0C8016FDA0E94F5120F900F900F9066
:104970000F90811103C080EE94E002C082ED94E0BC
:1049800041E065E18BD80E945F56BC016F5F7F4FAD
:10499000C8010E94B25A67E174E0C8010E94685AD7
:1049A0006BE174E0C8010E94685A0E945F56FC01E6
:1049B000808140E1BE016F5E7F4F90E00E94FE5A11
:1049C000BE016F5E7F4FC8010E94935A69E174E097
:1049D000C8010E94685A6EE1C80134DA0E945F562D
:1049E000FC0180894AE0B80190E00E94FE5A6DE126
:1049F00074E0C8010E94685A0E945F56FC018785D6
:104A000090E04AE0BE016F5E7F4F8053984F0E9456
:104A1000FE5ABE016F5E7F4FC8010E94935A67E243
:104A2000C8016DC10E94F512811103C084EC94E0AD
:104A300002C089EB94E041E060E030D80E945F560C
:104A4000FC01638574858585968520E1AE014F5F05
:104A50005F4F0E94085B69E0CE010196F3D90E9486
:104A6000F512811103C084EB94E002C08EEA94E059
:104A700041E069E113D80E945F56FC012189328927
:104A800043895489658976898789908D04E10E94DC
:104A9000195AE22FA42FF52F2AE0AE014F5F5F4F86
:104AA0006E2F732F8A2F9F2F0E94085B67E174E09F
:104AB000CE0101960E94685A0E94F512811103C02E
:104AC00064E274E002C061E274E0CE0101960E94EB
:104AD000685A62E212C10E94F512811103C080EA95
:104AE00094E002C082E994E041E060E00E944E1D43
:104AF0000E945F5669E00496A5D90E94F5128111C3
:104B000003C067E874E002C06DE774E0CE0101966F
:104B10000E94735A0E945F56FC01828540E1BE01EB
:104B20006F5E7F4F90E00E94FE5ABE016F5E7F4F26
:104B3000CE0101960E94935A62E1CE01019682D97C
:104B40000E94F512811103C085E794E002C08DE652
:104B500094E041E06BE10E944E1D0E945F56FC0113
:104B6000848D813059F028F0823069F08330A9F0CB
:104B7000C7C041E064E28EE594E01AC041E064E21F
:104B800082E594E015C00E94F512811103C088E40B
:104B900094E00CC08AE394E009C00E94F5128111F0
:104BA00003C082E394E002C087E294E041E064E263
:104BB0000E944E1DA5C00E94F512811103C08EEB0C
:104BC00093E002C087EB93E041E060E00E944E1D5D
:104BD0000E94E95690E080319105E8F4FC01E1592A
:104BE000FF4F0C942A5982E194E021C08FEF93E0AB
:104BF0001EC086EF93E01BC080EF93E018C08AEEE2
:104C000093E015C080EE93E012C086ED93E00FC0F4
:104C100089EC93E00CC00E94F512811106C082E37A
:104C200094E005C08CE094E002C087E294E041E0AB
:104C300069E00E944E1D0E94F512811103C081EBB4
:104C400093E002C089EA93E041E065E10E944E1DD5
:104C50000E94F512811103C06CE873E002C063E8A2
:104C600073E0CE0101960E94735A0E94D8564AE022
:104C7000BE016F5E7F4F0E94FE5ABE016F5E7F4F86
:104C8000CE0101960E94935A6EE1CE010196DAD8C8
:104C90000E94F512811103C06FE973E002C065E95B
:104CA00073E0CE0101960E94735A0E94C7564AE0F3
:104CB000BE016F5E7F4F8130F0E29F0750F40E948B
:104CC000FE5ABE016F5E7F4FCE0101960E94935A3D
:104CD00013C0892F8695869590E00E94FE5ABE01EA
:104CE0006F5E7F4FCE0101960E94935A6FE174E090
:104CF000CE0101960E94685A67E2CE010196A2D8C1
:104D00002091A60545E0249F90011124442737FDFA
:104D10004095542FEE24E39403E564E170E080E0D5
:104D200090E0D8CD0E94F512811103C002E416E094
:104D300002C00FE316E00E94F512811103C067E381
:104D400078E002C061E378E0A80180E00E94F71DEE
:104D50000E94F512811103C002E416E002C00FE3C5
:104D600016E00E94F512811103C062E276E002C0F3
:104D70006CE176E0A80181E00E94F71D0E94F51227
:104D8000811103C00CE316E002C008E316E00E94A4
:104D9000F512811103C060E376E002C068E276E0BC
:104DA000A80182E00E94F71D0E94F512811103C044
:104DB0000CE316E002C008E316E00E94F512811130
:104DC00003C065E176E002C06EE076E0A80183E012
:104DD0000E94F71D0E94F512811103C00CE316E03A
:104DE00002C008E316E00E94F512811103C067E0DB
:104DF00076E002C060E076E0A80184E00E94F71D42
:104E00000E94F512811103C00CE316E002C008E312
:104E100016E00E94F512811103C06BEF75E002C02D
:104E200064EF75E0A80185E00E94F71D0E948913D8
:104E3000813039F40E94F51281110AC00BE416E0AA
:104E40000CC00E94F512811106C005E516E005C0F0
:104E500005E416E002C000E516E00E94F51281119B
:104E600003C06CEE75E002C065EE75E0A80186E057
:104E70000E94211D0E94F512811103C06EED75E0A4
:104E800002C063ED75E04BE951E087E00E94211D0F
:104E90000E94F512811103C06BEC75E002C06EEB4D
:104EA00075E04BE951E088E00E94211D80918E055C
:104EB00081110BC06091A60589E0689F602D1124C7
:104EC00029E042E582E00E94510D00E020E342E04B
:104ED00060E080E00E94BC0C80918E05811167C467
:104EE000E9CC0E94F512811103C08FEA95E002C05F
:104EF00086EA95E041E069E00E944E1D0E94F512AD
:104F0000811103C08AE995E002C08FE895E041E095
:104F100062E17EC102E010E040E3410F61E0802FDA
:104F20000E94011641E4410F6AE0802F0E940116A1
:104F30004BE4410F63E1802F0E940116163018F4F4
:104F400045E5410F0DC0163051F0173021F01830F3
:104F500021F448E805C04FE503C047E801C04DE231
:104F60006CE1802F0E9401161F5F085F1A30A1F6C6
:104F70008091A605612F0E94B95869E0869F602D37
:104F8000112429E049E0892F880F880F880F0E949B
:104F9000510D41E867E280E00E94011645E955E0C5
:104FA00067E28E5F0E94A817182F0E94C41BFC01A5
:104FB0009681993120F09353983108F0F8C322E09C
:104FC00045E06DE2812F04C10E94C41B8C018091D9
:104FD000A60581110AC043E861E08DE00E94011638
:104FE00044E86DE08DE00E940116F801428167E01F
:104FF0008AE00E948D1C982F3BE0F32EF80E8091E2
:10500000A605811109C02BE04EE065E08DEF890F08
:10501000998F0E94510D998D4DE267E08CE0890FC8
:105020000E9401168F0D23E0E22EE80E9091A60556
:10503000913069F496E0F92EF80E43E861E08F2D87
:105040000E94011644E86DE08F2D0E940116F801C0
:10505000418167E08E2D0E948D1CE80EFF24F394A1
:10506000FE0C8091A605813039F42BE04EE065E01E
:1050700083EF8E0D0E94510D4DE267E082E08E0DB0
:105080000E940116F80EB3E0DB2EDF0C8091A6051E
:10509000823069F443E861E0ACE0EA2EEF0C8E2D3B
:1050A0000E94011644E86DE08E2D0E9401160E94B8
:1050B0009513F8012081AC01420F511D67E08D2D41
:1050C0000E944F1C9091A605923041F49AEE9F0DDC
:1050D0002BE04AE165E0890F0E94510D8091A60501
:1050E000833051F443E868E182E10E94011644E80C
:1050F00064E282E10E940116F80143816EE18FE0D3
:105100000E948D1CF0E1FF2EF80E9091A6059330C1
:1051100031F42BE04FE06CE18F5F0E94510D4AE3C8
:105120006EE18F2D0E9401168F0DFF24F394F80E6F
:105130009091A605943069F4E4E0EE2EE80E43E881
:1051400068E18E2D0E94011644E864E28E2D0E94D3
:105150000116F80144816EE18F2D0E948D1C8F0D88
:10516000FF24F394F80E9091A605943031F42BE0CF
:105170004FE06CE18E500E94510D4AE36EE18F2D9D
:105180000E940116F80EDD24D394DF0C8091A60551
:10519000853069F443E868E174E0E72EEF0C8E2D6A
:1051A0000E94011644E864E28E2D0E940116F80167
:1051B00045816EE18D2D0E948D1C9091A605953044
:1051C00009F0F5C293EF9F0D2BE04FE06CE1890FE2
:1051D0000E94510DECC260E085E995E00E94221F1B
:1051E0000E94F512811103C084E793E002C085E6B6
:1051F00093E041E062E10E944E1D0E94F512811190
:1052000003C089E593E002C08BE493E041E06BE1E9
:105210000E944E1D0E94F512811103C087E098E0A4
:1052200002C083E098E00E944A1C0E94F51281119E
:1052300003C08DE098E064C28AE098E061C20E94F9
:10524000F512811103C084E997E019C088E897E05E
:1052500016C00E94F512811103C082E892E002C0DC
:1052600089E792E041E069E00E944E1D0E94F5123C
:10527000811103C081E792E002C084E692E041E040
:1052800062E193C20E94F512811103C082E493E0AF
:1052900002C084E393E041E069E00E944E1D0E9459
:1052A000A413482F50E067E185E20E944F1C01E003
:1052B00028E040E460E28AE00E94BC0C78C20E94D0
:1052C000F512811103C08EE293E002C087E293E001
:1052D00041E062E00E944E1D2BE044E560E080E08A
:1052E0000E94510D80918C05833009F451C028F43F
:1052F000813049F08230F1F0ADC0843009F490C0C3
:10530000853079F1A7C00E94F512811103C08AE1AE
:1053100093E002C08AE093E041E060E10E944E1D0C
:105320000E94F512811103C085E093E08FC080E0F8
:1053300093E08CC00E94F512811103C085EF92E0CA
:1053400002C083EE92E041E060E10E944E1D0E94A7
:10535000F512811103C08EED92E078C089ED92E0E4
:1053600075C00E94F512811103C08DEC92E002C05D
:105370008BEB92E041E060E10E944E1D0E94F5122D
:10538000811103C086EB92E061C081EB92E05EC0C8
:1053900090913005892F827090FF16C0882351F0BC
:1053A0000E94F512811103C081E392E018C085E2EA
:1053B00092E015C00E94F512811103C088E192E0CD
:1053C0000EC089E092E00BC0882369F00E94F512BC
:1053D000811103C08BEF91E002C08CEE91E041E0BF
:1053E00060E10E944E1D4AE0BE016F5F7F4F8091D9
:1053F0002E0590912F050E94FE5A0E94F5128111F0
:1054000003C064EE71E002C06CED71E0CE01019664
:105410000E94685A69E1CE0101960E94221F1AC0BB
:105420000E94F512811103C086EA92E002C086E96B
:1054300092E041E060E10E944E1D0E94F512811150
:1054400003C08FE892E002C089E892E041E069E1A0
:105450000E944E1D01E020E344E560E080E00E94F0
:10546000000DA5C10E94F512811103C086E492E0EF
:1054700002C08DE392E041E062E00E944E1D6BE0CD
:1054800032C00E94F512811103C08CE592E002C087
:105490008EE492E041E062E00E944E1D2BE044E584
:1054A00060E080E00E94510D01E020E344E560E00F
:1054B00080E00E94000D41E060E183EA91E00E94FB
:1054C0004E1D41E069E18FE991E00E944E1D60911F
:1054D000A60589E0689F602D1124615F29E042E202
:1054E00089E176CE60E085E995E00E94221F5FC1E8
:1054F00060E085E995E00E94221F01E027E044E595
:105500006AE080E00E94000D0E94AB36882389F09B
:105510000E94C41BFC01F4800E94C41BFC01058195
:105520000E94C41BFC01F0820E94C41BFC01018389
:1055300008C00E94C41BFC01F0800E94C41BFC0137
:10554000018110E0FCE3FF9E000D111D11240E945B
:10555000C41B44E6409F9001419F300D1124FC0183
:105560008681A901480F511DCA010E943A3820E5E1
:10557000209FC001219F900D11246091930570918F
:1055800094050E94C558462F01E023E06CE082E0BC
:105590000E94BC0C8091BB07882309F447C00E947D
:1055A000F512811103C042EF57E002C04DEE57E003
:1055B00063E180E00E94C917182F8091AB07811129
:1055C0000BC04091BB0750E063E185E0810F0E9472
:1055D0004F1C195F180F1DC00E94C41BFC0186815F
:1055E000893138F09DEC980F81E0983118F080E017
:1055F00001C081E080FDE5CF8091BB078A3010F4C7
:10560000135F07C08091BB07843610F41D5E01C094
:10561000175E4FE263E1812F0E940116810F4091D6
:10562000BC0750E063E18E5F0E944F1C8091AB0786
:10563000882371F00E94F512811103C087E398E07E
:1056400002C081E398E041E06DE10E944E1D2EC052
:105650000E94AB36882389F00E94C41BFC01148190
:105660000E94C41BFC0105810E94C41BFC01108325
:105670000E94C41BFC01018308C00E94C41BFC01E2
:1056800010810E94C41BFC010181412F6DE18DE15D
:105690000E948D1C1DE1180F4AE36DE1812F0E94CD
:1056A0000116402F6DE1810F0E948D1C0E94AB36C8
:1056B000811104C08091AB07882329F10E94F51263
:1056C000811103C082E498E002C08DE398E00E945B
:1056D0004A1C8091AB07882351F00E94F51281117A
:1056E00003C08AE298E00CC08FE198E009C00E94F4
:1056F000F512811103C087E398E002C081E398E0CE
:105700000E94101D54C00E94F512811103C086EA48
:1057100097E002C08FE997E041E067E246C060E0B1
:1057200085E995E00E94221F0E94C41BFC010581AF
:1057300044816DE18DE10E948D1C1DE1180F4AE34B
:105740006DE1812F0E940116402F6DE1810F0E94B3
:105750008D1C40912E0550912F0569E080E00E943C
:105760004F1C0E94F512811103C082E498E002C030
:105770008DE398E00E944A1C1AC00E94F512811124
:1057800003C085ED91E002C08BEC91E041E060E167
:105790000E944E1D0E94F512811103C083EC91E01E
:1057A00002C086EB91E041E069E10E944E1D0E943B
:1057B00000366C96E2E10C94E3598F929F92AF927F
:1057C000BF92CF92DF92EF92FF92CF93DF93C82FD9
:1057D0004091400350E04931510508F0B3C7FA0148
:1057E000E158FF4F0C942A59823009F0ABC70E9450
:1057F000D709609388057093890580938A059093F3
:105800008B0561E975E085E995E00E94723888E0D2
:105810008093400397C70E94973BC0908805D09023
:105820008905E0908A05F0908B056C157D058E0545
:105830009F05B0F0C250C23008F084C78091300597
:10584000882351F083E080938C0581E0809381056B
:1058500083E18093400376C781E08093400372C761
:10586000C13009F442C078F1C23019F0C33009F1F7
:1058700069C70E943D3B60918405709185058091C8
:105880008605909187050E94835480913005882376
:1058900041F083E080938C0581E08093810583E172
:1058A00001C081E0809340030E948A510E948A5186
:1058B00049C70E94A03B811103C00E94523B42C7CE
:1058C0000E945D3B3FC70E94A03B882309F43AC772
:1058D0009091BB078091BC07981708F033C780915F
:1058E000BB078F5F8093BB072DC70E94A03B882317
:1058F00009F428C78091BB07823008F423C7809140
:10590000BB0781508093BB071DC7813091F028F001
:10591000C350C23008F016C717C08091A60588236F
:1059200021F081508093A6050DC784E08093A605E1
:1059300009C78091A605843020F48F5F8093A60567
:1059400001C71092A605FEC68091A60581110CC064
:10595000879906C081E0809340030E947F1EF2C6B3
:1059600081E180934003EEC6813041F48799F8CFFE
:1059700085E1809340031092A605E4C6823051F47D
:1059800084E0809340031092830510928205109268
:10599000A605D8C6833099F480E1809340030E9425
:1059A000651F879908C089E0809340031092A6057F
:1059B0000E94FB55C7C681E180934003C3C6843073
:1059C00009F0C0C685E080934003BCC61092400336
:1059D000B9C60E948A51FC0142815381648175815C
:1059E000452B462B472B19F40E948F1EABC6C111C5
:1059F00065C08091A60581115DC08091820590915E
:105A00008305009731F00197909383058093820579
:105A100099C60E948A51FC0186819781A085B18533
:105A2000892B8A2B8B2B09F48DC60E948A51FC018D
:105A300080809180969487940E948A51A12CB12CE9
:105A40002091820530918305FC0186819781A08594
:105A5000B185820F931FA11DB11D88169906AA0654
:105A6000BB06A0F40E948A512091820530918305E3
:105A7000FC01C680D780E084F184C20ED31EE11CF5
:105A8000F11CC818D908EA08FB0803C0C12CD12CA6
:105A900076010E948A51FC018681978101978C19B9
:105AA0009D099093830580938205C701B6010E94EA
:105AB000835448C681508093A60544C6C13009F07E
:105AC000A6C08091A605C0908205D0908305C80E1F
:105AD000D11CE12CF12C0E948A51FC01828193811E
:105AE000A481B5810197A109B109C816D906EA06B2
:105AF000FB0608F027C68091A605843020F48F5F4E
:105B00008093A6051FC6C0918205D09183050E948F
:105B10008A51FC01808191810597C817D90750F4FB
:105B200080918205909183050196909383058093DF
:105B3000820508C60E948A51FC01C680D780E08495
:105B4000F1840E948A51FC0180819181C80ED91E86
:105B5000E11CF11C0E948A51FC0182819381A48185
:105B6000B5810197A109B1098C159D05AE05BF0549
:105B700008F4E8C50E948A51FC01808091809694C7
:105B800087940E948A51A12CB12C209182053091DA
:105B90008305FC0186819781A085B185820F931FC3
:105BA000A11DB11D88169906AA06BB06A0F40E9485
:105BB0008A512091820530918305FC01C680D780EF
:105BC000E084F184C20ED31EE11CF11CC818D90870
:105BD000EA08FB0803C0C12CD12C7601C0918205D4
:105BE000D09183050E948A519E012F5F3F4FFC0197
:105BF00086819781280F391F2C193D093093830521
:105C000020938205C701B6010E9483549BC5C23010
:105C100049F40E948F1E811195C510924003109285
:105C2000A60590C5C33009F04DC00E94851DEC014A
:105C300088818E3379F480E1809340030E94651F50
:105C4000CE0101960E949C510E947F1E81E08093AC
:105C5000400378C50E948A510E948A51CE010E9459
:105C6000CD5A843008F46EC59E01280F311DF9010C
:105C7000349720812E3209F065C53196308130622B
:105C8000319620812062319680818062343739F4E8
:105C9000213609F057C5803709F054C586C5373716
:105CA00039F4213609F04EC5863709F04BC557C582
:105CB000323609F047C5213609F044C5873709F067
:105CC00041C5B9C5C43009F03DC50E94851D2EE00F
:105CD0002093400340E150E0BC0185E995E00E943B
:105CE000B95A30C581E0809340032CC5823009F059
:105CF00029C580918D05813019F40E94050A04C0E0
:105D0000823011F40E94DB0B1092400381E08093FB
:105D1000A60518C581E08093A605809130058823EB
:105D200049F083E080938C051092810583E1809394
:105D3000400308C51092400305C5813009F48EC0A8
:105D400008F477C0823019F0833041F0FBC48093AF
:105D5000A605109240030E94A714F4C42091A60542
:105D60008091820590918305820F911D8930910564
:105D700008F0E8C4FC01E856FF4F0C942A590E9431
:105D8000F51291E0811190E0892F0E94F912DAC496
:105D90000E94111391E089270E941713D3C40E9417
:105DA0001E1391E089270E942413CCC40E942B1358
:105DB00091E089270E942F13C5C40E9436138111D8
:105DC00004C081E00E943B13BDC40E9436138130A1
:105DD00021F482E00E943B13B5C480E00E943B1393
:105DE000B1C40E940113833021F480E00E940713A4
:105DF000A9C40E9401138F5F0E940713A3C48AE005
:105E00008093400310928E051092A6051092830590
:105E10001092820597C48DE0809340030E94C41BBA
:105E20000E94A41B1092A6058DC482E180934003BA
:105E300089C48091A605882321F081508093A6050E
:105E400081C48091820590918305009709F47AC4FA
:105E50000197909383058093820574C48091A60571
:105E6000843020F48F5F8093A6056CC480918205F6
:105E7000909183058430910508F064C40196909355
:105E80008305809382055EC4813009F4ADC008F4B7
:105E900074C0823019F08330A1F054C480918E0513
:105EA000882319F010928E054DC482E090E0909303
:105EB00083058093820584E08093A6058093400348
:105EC00041C480918205909183054091A6059C0173
:105ED000240F311D2630310509F442C060F027300F
:105EE000310509F446C02830310509F02BC48BE098
:105EF0008093400327C490918E05242F280F992367
:105F000021F180918F0590919005223099F038F41D
:105F1000222369F02130B1F40E94521313C02430BF
:105F200079F058F0253071F40E9484130BC00E9460
:105F30005C1308C00E94661305C00E94701302C063
:105F40000E947A1310928E05FDC3822F0E94C01DFD
:105F50009093900580938F0581E080938E05F2C326
:105F60000E94891391E0811190E0892F0E948E1385
:105F7000E9C387E080934003E5C380918E052091BB
:105F8000A6058823F1F080918F05909190050196E8
:105F90009093900580938F05E0918205F0918305A1
:105FA000E20FF11DEE0FFF1FED57FE4F25913491CB
:105FB0002817390708F0C6C33093900520938F0542
:105FC000C1C3222321F021502093A605BBC3809199
:105FD000820590918305009709F4B4C301979093CB
:105FE000830580938205AEC380918E052091A6051E
:105FF0008823F1F080918F059091900501979093FF
:10600000900580938F05E0918205F0918305E20F62
:10601000F11DEE0FFF1FE157FE4F259134918217BE
:10602000930708F08FC33093900520938F058AC3A0
:10603000243020F42F5F2093A60584C3809182052D
:10604000909183058430910508F07CC3019690936C
:1060500083058093820576C3823061F48AE0809361
:10606000400384E090E090938305809382058093C1
:10607000A60568C3833009F065C38AE080934003B6
:1060800084E090E090938305809382058093A60539
:106090000E94A71357C3882319F0813051F012C012
:1060A0008091A605882309F44DC381508093A605ED
:1060B00049C38091A605833008F044C38F5F809365
:1060C000A60540C383E08093A605109240033AC31F
:1060D000823059F028F48823D1F0813019F132C38D
:1060E000833061F0843051F12DC38091A60588235F
:1060F00009F428C381508093A60524C38091A60586
:10610000873208F01FC38F5F8093A6051BC3809161
:10611000A6058A508093A605853608F413C310920D
:10612000A60510C38091A605865F8093A6058832D8
:1061300008F408C387E28093A60504C385E995E0C7
:106140000E94CD5A9C015091A605563249F48823ED
:1061500009F4F8C2F901FF27EC56FA4F1082F2C297
:10616000573209F08FC0811106C081E08093A605E7
:1061700010924003E7C280918D05813019F461EBE4
:1061800071E009C0833019F46CEA71E004C0823018
:1061900031F467EA71E085E995E00E94685A89E187
:1061A000809340030E94651F0E9448090E94CC51C1
:1061B0000E94985385E995E00E940352882321F0BC
:1061C0008FE080934003BEC2C0918D05C130E1F4E1
:1061D00085E995E00E944D09811112C085E995E09D
:1061E0000E94CD5A99278F569A4FFC011082C09376
:1061F0008C058CE08093810583E180934003A2C2EB
:1062000087E0809340039EC2C330E1F485E995E0C6
:106210001FD4811113C085E995E00E94CD5A9927BA
:106220008F569A4FFC01108281E080938C058CE0A0
:106230008093810583E18093400384C287E080934B
:10624000400380C2C23009F07DC285E995E00E941A
:10625000680A811113C085E995E00E94CD5A9927FB
:106260008F569A4FFC01108281E080938C058CE060
:106270008093810583E18093400364C287E080932B
:10628000400360C28C3008F05DC23327EAE0852FFE
:106290006E2F0E94B958492F852F0E94B95881301E
:1062A00041F028F0823041F0833041F017C090E394
:1062B00001C091E4940F15C09BE4FCCF463010F46C
:1062C00095E5F8CF463061F0473021F0483021F4B1
:1062D00098E807C09FE505C097E803C090E001C0BB
:1062E0009DE2F901EB56FA4F908311822BC2823066
:1062F00069F030F4882319F1813009F461C022C2B9
:10630000833091F0843009F487C01CC224E02093CC
:10631000400383E090E0909383058093820520936F
:10632000A6050E94A7140EC28091A605853020F410
:106330008F5F8093A60506C21092A60503C28091C6
:10634000A605823001F50E949513EC010E94C41B42
:10635000FC018081C80FD11DC433F8E0DF0708F4C9
:1063600021960E949513C81BD90BC430D10518F192
:106370000E94951304960E949A130E94C41B2497AE
:10638000FC01C08318C0813029F030F0833051F017
:10639000CBE309C0CCE007C00E94C41B0E94C71B0E
:1063A000C82F01C0C7E10E94F11CFC0180818C173D
:1063B00010F48F5F80830E94C41B0E94B21BC2C175
:1063C0008091A6058230D9F40E949513EC010E94B9
:1063D000C41BFC018081C80FD11DC03EF7E0DF0760
:1063E00008F021970E949513C817D90728F40E9436
:1063F000951304970E949A130E94951308C00E9457
:10640000F11CFC012081222311F0215020830E94E5
:10641000C41B0E94B21B96C10E94C41BFC01858153
:106420008F3168F00E94C41B2BE3FC0125830E947E
:10643000C41B23E6FC0126830E94D71B04C00E94D4
:10644000C41BFC0115820E94C41B0E94B21B7AC1AE
:10645000823009F077C181E08093400373C18230BC
:1064600019F0833071F06EC185E995E00E94CD5A34
:1064700099278F569A4FFC0110828CE0809340033D
:1064800061C1C0918D05C130E1F485E995E00E94BC
:106490004D09882321F087E08093400353C185E9AB
:1064A00095E00E94CD5A99278F569A4FFC01108291
:1064B000C0938C058CE08093810583E18093400339
:1064C00041C1C23009F03EC185E995E00E94680AE9
:1064D000882321F087E08093400334C185E995E06B
:1064E0000E94CD5A99278F569A4FFC01108281E065
:1064F00080938C058CE08093810583E18093400339
:1065000021C1109240031EC10E94A413C13079F032
:1065100040F0C23099F0C33009F014C10E94A714B2
:106520000DC087FD0FC18F5F0E949F130BC1882391
:1065300009F408C181500E949F1304C18091A605EF
:10654000811103C010924003FDC084E0809340039A
:10655000F9C080918C05833031F410922F05109290
:106560002E05109230058091810580934003EAC08A
:106570008130E1F090F0823001F1833009F0E2C027
:106580008091A6058F5F80938D051092A6058CE003
:106590008093400310929505D5C08091A60588236D
:1065A00009F4D0C081508093A605CCC08091A60587
:1065B0008111C8C0C093A605C5C01092400381E0F8
:1065C0008093A605BFC08ED281E08093A6058091FE
:1065D0003005882349F083E080938C051092810573
:1065E00083E180934003AEC010924003ABC081E0D2
:1065F0008093A60580E00E94BB0B811109C085E055
:1066000080938C051092810583E1809340039AC0AA
:1066100080913005882349F083E080938C051092A7
:10662000810583E1809340038DC0109240038AC0AE
:10663000813009F47AC008F468C0823019F08330E0
:1066400001F180C088D3811137D3609184057091A6
:10665000850580918605909187050E9483548091DD
:106660003005882351F083E080938C0581E080938E
:10667000810583E18093400365C081E080934003FE
:1066800061C00E949E56811118C06091840570916E
:10669000850580918605909187050E94835480919D
:1066A0003005882339F0C0938C0581E08093810503
:1066B00083E101C081E0809340038091AB078111A9
:1066C00012C00E94C41BEC010E94C41BFC01848107
:1066D00088830E94C41BEC010E94C41BFC018581BD
:1066E000898347D42FC04FD40E94C41BEC010E9461
:1066F000C41BFC0180818C830E94C41BEC010E949E
:10670000C41BFC0181818D831DC025D381111AC05A
:106710009091BB078091BC079817A0F48091BB07AC
:106720008F5F8093BB073AD40DC015D381110AC087
:106730008091BB07823030F08091BB0781508093FD
:10674000BB072CD40E94651FDF91CF91FF90EF9083
:10675000DF90CF90BF90AF909F908F90089584E18D
:106760008093400341E150E0BE0185E995E00E943D
:10677000B95A0E94651FCE010E940418813049F465
:1067800092E090938C058093810583E18093400390
:10679000D9CF8230B9F684E080938C0581E0809374
:1067A000810583E180934003CDCF0E948A51FC0193
:1067B0004681578160857185409384055093850596
:1067C000609386057093870580E1809340030E9463
:1067D000651F61E975E0CE0185D480919205813015
:1067E00049F482E080938C051092810583E18093C7
:1067F0004003A8CF882321F086E080934003A2CFF6
:1068000082E080934003CE010E940F5441E150E0AA
:10681000BE0185E995E00E94B95A0E94FA51609341
:1068200088057093890580938A0590938B05BDD662
:106830000E94411C87CF80E1809340030E94651F26
:10684000CE018DD290939405809393050296029782
:1068500050F482E080938C0581E08093810583E190
:10686000809340036FCF41E150E0BE0185E995E0A0
:106870000E94B95ACE0129D20E94411C87E180931F
:10688000400360CF8091400390E0FC013297E731F4
:10689000F10508F061C0EF55FF4F0C942A59809123
:1068A0003F038F5F80933F038530D8F455C08091BC
:1068B0003F038F5F80933F03893198F408950E94CE
:1068C0002F0A90913F03813039F4943609F444C083
:1068D00084E680933F033EC09F5F90933F039530D3
:1068E000D8F110923F0336C080918D05813051F46C
:1068F0000E942C0AFC018081882321F083E0809390
:10690000400328C080918D05823031F50E94DE0B56
:10691000882311F188E1809340030E94C41BFC018D
:10692000148215820E94651F0C949E0A089580911E
:106930008E05882379F080E00E94F715882311F0F6
:1069400080E006C081E00E94F715882319F081E0FD
:106950000E94DD2B0C94651F0895843508F083E5B3
:10696000443508F043E5603308F06FE2203308F067
:106970002FE2E091A507F091A6079081891708F40E
:1069800080838281841708F442838181681708F428
:1069900061838381821708F423830895E091A5071A
:1069A000F091A60783E5808312828FE281831382B0
:1069B000089548EF51E060E070E08091A307909166
:1069C000A4070E948C5A2FE243E560E080E0C5DF17
:1069D00017C1089548EF51E060E070E08091A3078F
:1069E0009091A4070E948C5A2FE243E560E080E07A
:1069F000B4CF08959093A4078093A3077093A6073C
:106A00006093A50708952AB53BB5809173059091D1
:106A10007405820F931F9BBD8ABD849B02C081E0D9
:106A200001C08FEF0E946B528091A7079091A80739
:106A3000A091A907B091AA070196A11DB11D80934D
:106A4000A7079093A807A093A907B093AA07089552
:106A5000A2E0B0E0EEE2F5E30C94D55989839A8385
:106A60000E94480989819A810E944554082F8823F1
:106A7000A1F11CE280E00E946B521150D9F70E94F4
:106A800071521092A7071092A8071092A9071092AE
:106A9000AA071FBC209105013091060140E050E09B
:106AA00060E074E284EF90E00E94EC58309374054B
:106AB000209373051DBC1CBC209173053091740597
:106AC0003BBD2ABD23E035E330937705209376055F
:106AD00097B7906197BF81E08EBD802F2296E4E04A
:106AE0000C94F15987B78F7E87BF0E94F5500E94A2
:106AF000715260E070E0CB010E94FA5262E579E4E5
:106B000086E496E40E94B1066091A7077091A807F9
:106B10008091A9079091AA076C5D7F4F8F4F9F4F7F
:106B20000E94B10667E571E486E595E40E94B1062E
:106B300066E67DE684E790E20E94B10660E170E0DF
:106B400080E090E00E94B10681E090E00E94AB06F8
:106B500081E090E00E94AB06609105017091060112
:106B600080E090E00E94B1066091050170910601FD
:106B700080E090E00E94B10681E090E00E94AB06C8
:106B800088E090E00E94AB0664E671E684E791E657
:106B90000E94B1066091A7077091A8078091A9078C
:106BA0009091AA070E94B1060E9471520E94C5529C
:106BB00081E008950F939093690580936805609331
:106BC0006A0540936B0520936C0500936D05109248
:106BD0006E050F910895C4980C94591A0895C49A9B
:106BE0000C94591A0895CF93C82F81E2F4DF8C2FAB
:106BF0008068F1DF80E2EFDF8CE0EDDFCF91089578
:106C0000EF92FF920F931F93CF93DF93C0E0D0E0FA
:106C100080E090E0E12CE091A507F091A6078C01BF
:106C2000085F1F4F218130E0201731073CF0E394CB
:106C3000CC5ADF4F0033110581F505C0238130E0C8
:106C40002817390734F4AADECDB7DEB7E6E00C9496
:106C5000EF598E2D8064BFDFE091A507F091A60764
:106C600080818068B8DFE091A507F091A607F080E9
:106C7000E091A507F091A60782818F15C0F20E94CE
:106C80000E0AE091A307F091A407EC0FFD1FEF0D92
:106C9000F11D8081A4DFF394EBCFC801BCCF0E942B
:106CA000621A81E298DF82E196DF80ED94DF80E274
:106CB00092DF8CE090CF089587B78F7E87BF1092C8
:106CC00084001B980C94C5520895CF92DF92EF92E6
:106CD000FF920E940F548823C1F10E949A560E948D
:106CE0009906623477458144964519F0E5DF82E0E4
:106CF0002DC00E948F060E948F061FBC1DBC1CBCAD
:106D00006C01E12CF12CA0EEBFEFA70196010E94CF
:106D10004B597C5D8B409F4F0E94EC583BBD2ABD78
:106D20008AB59BB58CEF97E09093770580937605B5
:106D30001092AC0791E09093BB071092AB0787B716
:106D4000806187BF9EBD80E001C081E0FF90EF9031
:106D5000DF90CF90089587B78295817008954F9204
:106D60005F926F927F928F929F92AF92BF92CF92DB
:106D7000DF92EF92FF921F93CF93DF93A8950E942B
:106D80000F54882309F4BFC00E94990662347745E6
:106D90008144964509F0B2C00E948F06029708F020
:106DA000ADC00E948F06EC01C13583ECD80708F016
:106DB000A5C061E070E080E090E00E942753882346
:106DC00009F49CC00E948856811132C081E08093F2
:106DD000BC0768E070E080E090E00E94FA528823EF
:106DE00009F48CC0C12CD12C7601A8950E9488563C
:106DF000882331F08F77C80ED11CE11CF11CF5CF30
:106E00000E94C5529E0140E050E0C701B6010E94B9
:106E1000EC5869017A01CA01B9012EEB30E040E07B
:106E200050E00E94EC582C0D3D1D4E1D5F1D64C0AE
:106E30008093BC079CE0899FB00111246F5F7F4F56
:106E4000882777FD8095982F0E942753882309F47F
:106E500055C010E0C12CD12C76019AE0492E512C5E
:106E6000612C712C8091BC07181730F50E9499068F
:106E70000E9499060E9499064B015C012EEB30E0BE
:106E800040E050E00E94EC58280D391D4A1D5B1D62
:106E9000C20ED31EE41EF51EC12FD0E0CC0FDD1FA5
:106EA000C950D64FCA01B901A30192010E94EC5802
:106EB000398328831F5FD6CF8091F7099091F80915
:106EC000A0E0B0E08093AD079093AE07A093AF072A
:106ED000B093B0078091AD079091AE07A091AF0736
:106EE000B091B0070E94C552C701B60128EE33E049
:106EF00040E050E00E94EC58C90107C00E94C55212
:106F00008FEF9FEF02C08EEF9FEFDF91CF911F9128
:106F1000FF90EF90DF90CF90BF90AF909F908F90B9
:106F20007F906F905F904F900895CF932091BC0712
:106F300030E0281B31092F5F3F4F8CE0829FB0016A
:106F4000839F700D11246F5F7F4F80E090E00E945F
:106F50002753811102C0C0E009C00E9499060E9417
:106F6000FA52C82F8823B9F30E9423528C2FCF9155
:106F7000089587B78F7E87BF109284001B9881E0A9
:106F80008093AB0708958091BB07CFDF882329F05A
:106F900097B7906197BF1092AB070895CF92DF9299
:106FA000EF92FF921F93CF93DF936091BC078CE029
:106FB000689FB00111246F5F7F4F882777FD809510
:106FC000982F0E942753182F882309F44AC0C1E044
:106FD000C12CD12C76018091BB078C17D8F00E9470
:106FE00099060E9499060E9499062091BB076C0D94
:106FF0007D1D8E1D9F1DC21718F46B017C0108C0FA
:107000006093AD077093AE078093AF079093B0077E
:10701000CF5FE1CFC701B60128EE33E040E050E09A
:107020000E94EC58E9010E94C41BFC01CE016CE3F4
:1070300070E00E94C558C82F64830E94C41BFC01E5
:10704000C5830E94C41BEC010E94C41BFC01848107
:1070500088830E94C41BEC010E94C41BFC01858133
:107060008983812FDF91CF911F91FF90EF90DF9067
:10707000CF9008952091AB07211133C04091AD0707
:107080005091AE076091AF077091B007A0E0B0E0FB
:1070900084179507A607B70720F1E091BB078091F9
:1070A000BC07E817F0F4EF5FE093BB078091AD07F2
:1070B0009091AE07A091AF07B091B007F0E0EE0F4E
:1070C000FF1FEB50F64F20813181820F931FA11DCE
:1070D000B11D8093AD079093AE07A093AF07B09317
:1070E000B0070895A0E0B0E0E8E7F8E30C94C759D2
:1070F000EB01198218821092BC071092940510922D
:1071000093050E940F54882339F0C12CD12C7601AD
:10711000412C512C32015BC081E08983D0C00E9498
:107120008856B82E0E948856082F22E0420E511C25
:10713000611C711C882309F453C00E94FA51641524
:1071400075058605970508F44DC0A89510E0102F29
:1071500000270B0D111D0E94FA514801A12CB12CE2
:107160006419750986099709681579058A059B05CB
:10717000D8F18091BC078F5F8093BC075301420117
:10718000312C01501109C401841995098017910708
:1071900098F40E948856282E3FEF831A930AA30A78
:1071A000B30A0E94FA51681579058A059B05F8F41F
:1071B0000E94FA5142E049830E9488562401350119
:1071C0002FEF421A520A620A720A381223C00E9432
:1071D000FA51461657066806790608F4A0CF23C070
:1071E000B110ABCF0E94FA5182E089831CC03224D7
:1071F00088E027FC06C05FEFC51AD50AE50AF50A44
:1072000005C092E0C90ED11CE11CF11C220C81507A
:1072100081F7B9CF88818111DACF33E0398380914A
:10722000BC078883D4CF0E945713EC010E944D13F2
:107230008C010E946B135C010E9475136091BC0766
:107240009C012A0D3B1DC00FD11F48EE53E0C49F87
:10725000C001C59F900DD49F900D1124280F391F98
:10726000629F4001639F900C1124A12CB12C0E94BD
:107270007F13A7019601220F331F441F551FDC0106
:107280000E943F59860E971EA81EB91E0E94011328
:10729000A501940104C056954795379527958A9581
:1072A000D2F7CA01B90120E432E44FE050E00E9475
:1072B000EC5830939405209393050E94C552CDB7A6
:1072C000DEB7E2E10C94E359A0E0B0E0EAE6F9E3CE
:1072D0000C94D259D62E0E940F54E82E882309F41C
:1072E0004FC00E945D531092B1071092B2071092E6
:1072F000B3071092B407F12CFD1409F441C00E94A9
:107300001D52182F0E941D524091B1075091B20793
:107310006091B3077091B4074E5F5F4F6F4F7F4F1F
:107320004093B1075093B2076093B3077093B407CB
:10733000C82FD0E0DC2FCC27C10FD11D00E010E01A
:107340000C171D07D9F00E941D524091B1075091B2
:10735000B2076091B3077091B4074F5F5F4F6F4FF3
:107360007F4F4093B1075093B2076093B307709378
:10737000B4070E945D530F5F1F4FE2CFF394BCCF61
:107380008E2DCDB7DEB7E7E00C94EE59A0E0B0E06B
:10739000ECECF9E30C94D1598091B6079091B707C2
:1073A000A091B807B091B907892B8A2B8B2B09F4D0
:1073B000D9C08091C007843029F08091C007873000
:1073C00009F0D0C08091BB0781116BC084E080932D
:1073D000C0070E941D52C82F0E941D524091B10744
:1073E0005091B2076091B3077091B4074E5F5F4F41
:1073F0006F4F7F4F4093B1075093B2076093B3072D
:107400007093B407282F30E0322F22272C0F311D24
:107410004091B6075091B7076091B8077091B907CE
:10742000C9010296481B590B610971094093B607BF
:107430005093B7076093B8077093B9078091BB0763
:107440008F5F8093BB0783B7846083BF12BE87B70B
:10745000816087BF3093BF072093BE070E944D1302
:107460008C010E946113EC010E940113F82E980117
:10747000A8EEB3E00E9430599E0140E050E00E9427
:107480000E590F2C04C056954795379527950A94A9
:10749000D2F73093C4072093C3071092C00712BEDF
:1074A0007FC08091C007873009F490CF0E945713A6
:1074B000EC010E9401139E0102C0369527958A9522
:1074C000E2F7C9016AE070E00E94C5587B010E94A2
:1074D000C41BEC014C813D812E8180E797E1489FE0
:1074E0008001499F100D112454E6359F000D111D98
:1074F0001124020F111D2E81F0E7CF2EF7E1DF2EB0
:107500005C814D813E815C9DC0015D9D900D11248B
:1075100054E6459F800D911D1124830F911D801B02
:10752000910B8E159F0548F48E81821749F3A8951B
:107530000E947015A7D92E81E3CF8091C0078630B5
:1075400079F18091C007853059F18091B60790910B
:10755000B707A091B807B091B907892B8A2B8B2B5D
:10756000F9F034CF8091B6079091B707A091B80792
:10757000B091B907892B8A2B8B2B91F48091C0078E
:10758000843021F08091C007873051F40E94C552A9
:107590000E941E1381111092840085E08093C00721
:1075A000CDB7DEB7E8E00C94ED59CF931092BB074E
:1075B00084E08093C0071092B1071092B207109236
:1075C000B3071092B4070E94FA516093B607709304
:1075D000B7078093B8079093B9070E940113C82F8B
:1075E0000E94611396958795969587950C2E02C0FB
:1075F000969587950A94E2F7282F20952093C10746
:107600000E946B1396958795969587950C2E02C0D0
:10761000969587950A94E2F7282F20952093C20724
:107620000E94751396958795969587950C2E02C0A6
:10763000969587950A94E2F7282F20952093BD0709
:107640000E947F139695879596958795AC010C2E91
:1076500002C0569547950A94E2F740954093B507C6
:107660009C01220F331F02C036952795CA95E2F779
:1076700020952093C507CF91089585E08093C0079A
:107680001092B6071092B7071092B8071092B90778
:107690000E941E138111109284001092BA070C945C
:1076A000C552089586E08093C0070E941E13811181
:1076B000109284001092BA070895A0E2B0E0E3E6C9
:1076C000FBE30C94D5590E94F555BC01CE010196FF
:1076D0000E94B25A0E94C5528091BB07882329F0AC
:1076E0008091BB0781508093BB076091BB07CE019F
:1076F0000196EADD0E94FA510091B1071091B2079C
:107700002091B3073091B407601B710B820B930B70
:107710006093B6077093B7078093B8079093B90743
:1077200087E08093C007A096E4E00C94F159609143
:10773000B1077091B2078091B3079091B407089593
:107740009091C00781E0963009F080E0089512BE64
:107750008091C007843010F01B9808958091BA077B
:10776000882361F01B9A0E941E13882321F08091C8
:107770000701809384001092BA0709C01B980E94E9
:107780001E1381111092840081E08093BA078091CA
:10779000C007811115C08091C10782BF8091C307C6
:1077A0009091C407892B51F08091C3079091C40731
:1077B00001979093C4078093C30702C081E008C07B
:1077C0008091C007813039F48091C20782BF82E086
:1077D0008093C00708958091C007823081F4809122
:1077E000BD0782BF83E08093C00780E1809344039C
:1077F0001092430310924203109241030895809126
:10780000C007833009F049C080914403803178F18A
:107810008091BE079091BF072091410330914203B0
:107820002817390710F084E0D3CF109244030E9448
:107830001D52809343038091B1079091B207A091AC
:10784000B307B091B4070196A11DB11D8093B10794
:107850009093B207A093B307B093B407809141030C
:10786000909142030196909342038093410380914B
:10787000430387FF03C08091C50702C08091B5070D
:1078800082BF9091440390FF05C080914303880F0D
:10789000809343039F5F909344030895A4E0B0E076
:1078A000E4E5FCE30C94CB594C01CB01BA01811403
:1078B000910409F476C0623071058105910508F4E0
:1078C00070C0D401ED91FC912085608071802B30D7
:1078D00089F524E030E040E050E00E94A059F40136
:1078E000A284B384C484D584E684F7840089118992
:1078F0000E94355AF4E0EF2EF12C8E010F5F1F4FDE
:10790000F3010995882309F44CC049815A816B81A0
:107910007C81411551056105710509F442C0DB0107
:10792000CA01805F9F4FAF4FBF404097A105B1058F
:10793000A0F537C022E030E040E050E00E94A059BE
:10794000D4011A96AC901A971B96BC901B971C9664
:10795000CC901C971D96DC901D971E96EC901E9760
:107960001F96FC901F9750960C91509751961C9122
:107970000E94355AE2E0EE2EF12C8E010F5F1F4F70
:10798000F3010995882369F089819A81AC0160E04F
:1079900070E001978F3E9F4F20F4342F252FCB01AD
:1079A00004C030E020E080E090E0632F722F249646
:1079B000EEE00C94E759A2E1B0E0E1EEFCE30C94B8
:1079C000C7591C012A013B01009709F4F6C0423057
:1079D00051056105710508F4F0C0D1011A96BC91FA
:1079E000BD83F101F385FE83D1011C96BC91BF8359
:1079F000F101F585F887D1011E96BC91B987F10197
:107A0000F785FA87D1015096BC91BB87F101F189C6
:107A1000FC87D101ED91FC9180858B3009F0A5C0E8
:107A2000C301B20124E030E040E050E00E94A059E0
:107A3000AD80BE80CF80D884E984FA840B851C8514
:107A40000E94355A2D873E876A016F87788B898B14
:107A50009A8BD101ED91FC910190F081E02D04E031
:107A6000E02EF12C8E010F5F1F4F0995882309F43A
:107A7000A4C089809A80AB80BC8081149104A10449
:107A8000B10409F498C0D501C401805F9F4FAF4F86
:107A9000BF400897A105B10508F48FC0D501C40106
:107AA000885F9F4FAF4FBF400897A105B10518F4FD
:107AB000812C912C5401F10186A597A5A0A9B1A90B
:107AC000892B8A2B8B2B21F446A657A660AA71AA74
:107AD00019821A821B821C82D101ED91FC910480D3
:107AE000F581E02D14E0E12EF12C8E010F5F1F4F88
:107AF0002D853E85A6016F85788989899A890995A2
:107B000081149104A104B10409F455C02401350184
:107B100087CF49805A804114510409F44CC0C201F6
:107B20004096089708F449C0B8EF4B16BFEF5B06C4
:107B300010F0412C512C1A821982D101ED91FC9147
:107B40000480F581E02DA2E0EA2EF12C8E010F5F7A
:107B50001F4F9301A401B501C6010995612C712C39
:107B6000411451046104710431F1C301B20122E0F6
:107B700030E040E050E00E94A059AD80BE80CF8050
:107B8000D884E984FA840B851C850E94355A390112
:107B90004A015B016C01D101ED91FC910190F081F2
:107BA000E02DB2E0EB2EF12C8E010F5F1F4F0995F7
:107BB0008111AFCF02C081E001C080E06296E2E1B6
:107BC0000C94E359A9E2B0E0E8EEFDE30C94C75948
:107BD0004C014CA35DA36EA37FA30B871C872D874D
:107BE0003E87009709F42FC1DC01ED91FC911197BC
:107BF0002081318139A728A7448155815A8B498B2F
:107C00001A965C911A975B8B1B968C911B978C8BA9
:107C10001C969C911C979D8B1D96AC91AE8BD401AC
:107C20001E96BC91BF8BD4011F96BC91B88FD40116
:107C30005096BC91B98FD4015196BC91BA8FD401A2
:107C40009E964D905D906D907C90D197B1E0BBA3D6
:107C50002085F40182899389A489B5892B3041F06C
:107C60001BA29C01AD01569547953795279509C0F4
:107C70009C01AD0192E056954795379527959A95C9
:107C8000D1F72B8F3C8F4D8F5E8FD4019E961D9226
:107C90001D921D921C92D1972B8D3C8D4D8D5E8D2A
:107CA0002F8F38A349A35AA31F82188619861A86D4
:107CB0008F8D98A1A9A1BAA1892B8A2B8B2B09F4AE
:107CC00061C032E0431651046104710448F08B8DA9
:107CD0009C8DAD8DBE8D481659066A067B0628F030
:107CE00082E0482E512C612C712C9BA1992329F103
:107CF000C301B20124E030E040E050E00E94A0590E
:107D0000AB88BC88CD88DE88EF88F88C098D1A8D09
:107D10000E94355A19014F87588BD62EC72EB82E80
:107D2000A92E04E0E02EF12C8E010F5F1F4FE8A575
:107D3000F9A50995811191C086C0C301B20122E065
:107D400030E040E050E00E94A059AB88BC88CD886C
:107D5000DE88EF88F88C098D1A8D0E94355A19013A
:107D60004F87588BD62EC72EB82EA92E12E0E12EA3
:107D7000F12C8E010B5F1F4FE8A5F9A50995811124
:107D8000BBC061C02B853C854D855E85232B242B94
:107D9000252B09F052C08CA19DA1AEA1BFA10297D5
:107DA000A105B10508F454C09BA1992319F12F81B5
:107DB000388549855A8529833A834B835C836CA136
:107DC0007DA18EA19FA124E030E040E050E00E9420
:107DD000A059AB88BC88CD88DE88EF88F88C098DE7
:107DE0001A8D0E94355AF4E0EF2EF12C8E010F5FB0
:107DF0001F4F1EC02F8138853E832D836CA17DA12E
:107E00008EA19FA122E030E040E050E00E94A05906
:107E1000AB88BC88CD88DE88EF88F88C098D1A8DF8
:107E20000E94355AE2E0EE2EF12C8E010B5F1F4FBF
:107E3000E989FA89099581110BC04F8158856985B7
:107E40007A85C401B8DD60E070E080E090E092C027
:107E50006F81788589859A858DC089819A81AB816A
:107E6000BC81892B8A2B8B2B09F05AC02B853C8532
:107E70004D855E85232B242B252B09F449C02F81AA
:107E8000388549855A85232B242B252B49F48FEFE0
:107E90009FEFAFEFBFE089839A83AB83BC8308C0B9
:107EA0002F81388549855A8529833A834B835C83A2
:107EB000B4E0EB2EF12C8E010F5F1F4F91014F8527
:107EC00058896D2D7C2D8B2D9A2DE989FA8909957C
:107ED000882309F4B2CF2B853C854D855E852150E2
:107EE0003109410951092B873C874D875E874F82B5
:107EF000588669867A8614C08D819E81892B81F48B
:107F00008B859C85AD85BE85892B8A2B8B2BD1F4E7
:107F1000D4019E964D925D926D927C92D1973BCF0B
:107F20002F8D38A149A15AA1215031094109510988
:107F30002F8F38A349A35AA33FEF431A530A630A6A
:107F4000730AB6CE2F81388549855A85232B242B79
:107F5000252B29F44FEF5FEF5E834D8304C08F81A3
:107F600098859E838D83A2E0EA2EF12C8E010B5F13
:107F70001F4FA4CFA996E2E10C94E35980E190E071
:107F80000895A0E0B0E0E7ECFFE30C94CF59EC01DA
:107F90000097E1F04230510561057105B8F0CB0161
:107FA000BA016250710981099109288D398D40E02B
:107FB00050E00E94A059AA8CBB8CCC8CDD8CEE8C3E
:107FC000FF8C08A119A10E94355A08C020E030E0BA
:107FD00040E050E060E070E080E090E0CDB7DEB7D8
:107FE000EAE00C94EB59FC01819191E080FB8795CC
:107FF00087F92191820F9F5F9B30C1F70895A0E020
:10800000B0E0E5E0F0E40C94D1598C01F701C480B4
:10801000D580C0E0D0E0C8018C0F9D1FCC15DD05D8
:1080200098F40E940051892B69F4F7014081518135
:10803000628173814F5F5F4F6F4F7F4F40835183EA
:10804000628373832296E7CF81E0CDB7DEB7E8E0A5
:108050000C94ED59ADE0B0E0E0E3F0E40C94C959C4
:108060006C0149012A013B01D701AD90BC901197E9
:1080700012968D919C911397809613969C938E9354
:108080001297F6018081853E11F0811104C0D7015D
:1080900014961C924FC0F60183858F3009F04CC0B6
:1080A000D70114968C91882319F095858917A9F02A
:1080B00045E350E060E070E0C5010E948C5AF60193
:1080C0008585D70114968C93F50105A716A787A679
:1080D00090AA41AA52AA63AA74AAD6018C918F735E
:1080E00090E001974DE0489F9001499F300D112489
:1080F000E8E0F1E0DE01119601900D924A95E1F77A
:10810000FE013196A20EB31EAE01425F5F4F2E1BE1
:108110003F0BC9018E0F9F1F4F9760F48191B601ED
:10812000680F711DDB018C91D5018D935D01E41702
:10813000F50779F781E0A9C0F5018081882341F036
:10814000C60151DFD70114969C91981709F459C0C4
:1081500045E350E060E070E0C5010E948C5AF501F3
:1081600005A716A787A690AA41AA52AA63AA74AA2D
:10817000D601A50180E09C91903299F0FA0190839C
:10818000F601248523FF07C02C9121542A3118F4CD
:10819000905EFA0190838F5F11964F5F5F4F88303A
:1081A00051F7D5019C91953011F495EE9C93F60111
:1081B0009085903211F1F501E80FF11D9EE2908358
:1081C000F601389634E0380F8F5F90819032A9F035
:1081D000A501480F511DDA019C93D6011C962C91E4
:1081E00024FF07C0208121542A3118F4905EDA015F
:1081F0009C938F5F31968313E8CFF501E80FF11D53
:108200001082F6018385D50190968C93C6014A961B
:108210000E9400512C01612C712CF50145A256A23F
:1082200067A270A6C60144960E940051AC0160E0AE
:1082300070E0BA0155274427442955296629772932
:10824000D50195964D935D936D937C939897C60158
:108250004C960E940851F50161A772A783A794A7C5
:10826000C60146960E940051D50192969C938E932A
:108270009197C60148960E940051F50194A383A3EB
:1082800081E0D70115968C9380E02D96E0E10C9467
:10829000E559A0E0B0E0EFE4F1E40C94D1598C0191
:1082A000F701C480D580C0E0D0E0C8018C0F9D1FCD
:1082B000CC15DD05A8F40E940851672B682B692BAB
:1082C00069F4F70140815181628173814F5F5F4F93
:1082D0006F4F7F4F40835183628373832496E5CF32
:1082E00081E0CDB7DEB7E8E00C94ED59AAE2B0E04A
:1082F000ECE7F1E40C94C7596C014B01009711F4C1
:1083000080E089C161157105D9F3CE0181967C01A8
:108310008E010E5D1F4F9E012D5D3F4FAE014C5DE6
:108320005F4FBE016B5D7F4F80970E94191C2981B2
:108330003A812C5B3740322F2227330F8DA1A0E2E8
:108340008A9FC0011124282B392B8CA1282BF401E2
:1083500034A323A32AA1F0E22F9F900111248BA123
:1083600090E0982F8827990F990F990F282B392B78
:1083700089A18695282BD40192963C932E939197B0
:10838000D601ED91FC91848195819AA789A7D401AA
:108390009D96BC91BEA3F401F6A5FFA3D4019F96C0
:1083A000BC91B8A7F40160A851A842A833A824A89A
:1083B000C4010E94CD5A6C01182F99270C966DE0CC
:1083C00070E00E94D958762E4BE050E060E270E0F9
:1083D000CE0101960E948C5A6EE270E0C4010E94A8
:1083E000F35A0097C9F0DC0111962C912223A1F0D9
:1083F0005C01BFEFAB1ABB0AC5010E94CD5A1FEF4B
:108400001C0D181B482F843008F043E050E0B501E4
:10841000CE0109960E94835A193098F4412F50E0FA
:10842000B401CE0101960E94835AF40180818E32FC
:1084300011F581818E3209F4828181111CC0712C69
:108440001AC048E050E0B401CE0101960E94835A60
:10845000D40195968C91982F92959F70803A10F444
:10846000905D01C09F599F838F708A3010F4805DAA
:1084700001C08F5988878981853E11F485E0898301
:1084800045E150E060E070E0CE010C960E948C5A0D
:10849000F40180A18C8761A172A1CE0147960E9450
:1084A0001751D40193966D917C919497CE01499682
:1084B0000E941751F40185A196A1A7A1B0A5BD0105
:1084C00088279927CE0145960E941751D401959689
:1084D0006D917C919697CE014B960E941751F401B5
:1084E00041A552A563A574A5CE014D960E941B51CE
:1084F000F0E27F9EA00111249A0140E050E060E08C
:1085000070E080E090E0AEA0BFA0C8A4D62CE52C1F
:10851000F42C032D122D0E94355A00E2E02EF12C8E
:108520008E010F5F1F4FE9A5FAA50995882309F46D
:10853000E7CEC80158DDC82ED72CADE0BA2EBFE07B
:10854000AB2EDD2009F461C040E250E06FEF70E037
:10855000CE0101960E948C5A8D2D90E00197B89E15
:10856000F001B99EF00D1124E80DF91D81E021E024
:10857000280F9191A1E0B0E0AC0FBD1FA80FB11D75
:108580009C938E5FA1E0B0E0AC0FBD1FA20FB11DA8
:108590001C928B3019F08A31D1F102C08EE038C0C4
:1085A000992311F08F3118F3D982D71003C08D2D84
:1085B00080648983AC86CE861D861B8E1C8EF0E27D
:1085C000EF2EF12C8E010F5F1F4F2EA13FA148A56A
:1085D000562D652D742D832D922DE9A5FAA50995AB
:1085E0002EA13FA148A5562D652D742D832D922DCA
:1085F000A0E20E943E5A2EA33FA348A7652E562E06
:10860000472E382E292EDA949CCF81E004C08CE1CD
:108610009111ADCFC9CFAA96E2E10C94E359A2E142
:10862000B0E0E5E1F3E40C94C9598C014230510506
:108630006105710548F1A5DC2A013B014C0140E1CF
:1086400050E060E070E0CE010196298B3A8B0E94E9
:108650008C5AD801ED91FC9111975896ED90FC90B1
:1086600059970680F781E02DA12CB12C5EEBC52E29
:108670005FE3D52E8E010F5F1F4F29893A89A20132
:10868000B301C401099501C080E06296E0E10C9459
:10869000E559A0E2B0E0EFE4F3E40C94C7591C0103
:1086A0004B01CA012114310409F470C1009709F487
:1086B0006DC10E94CD5A0C966DE070E00E94C558C5
:1086C0006F5F68A3D4014D905D906D907C90D10157
:1086D000ED91FC911197808541145104610471045E
:1086E000E9F58B3039F49A964D905D906D907C90C1
:1086F0009D9734C0F101F2A1FA83D1019396BC9108
:10870000BB83F101F4A1FC83D1019596BC91BD839B
:10871000F101F6A1FE83D1019796BC91BF83F101CF
:1087200080A491A4F28DF88FD1015B96BC91B98F92
:10873000F101F48DFA8FD1015D96BC91BB8FF101EF
:10874000F68DFC8FD1015F96BC91BD8FF101F0A138
:10875000FE8FD1019196BC91BF8F10C0188E198EDB
:108760001A8E1B8E1C8E1D8E1E8E1F8E1A821B82D1
:108770001C821D821E821F82812C912CEA81E88B33
:10878000FB81F98B0C810A8B1D811B8B2E812C8B1D
:108790003F813D8B8E8A9F8A18862A813B814C813E
:1087A0005D816E817F81C401A88CB98CCA8CDB8C01
:1087B000EC8CFD8C0E8D1F8D0E94535A09F08FC0DA
:1087C000411451046104710409F4E0C0A0E00E9466
:1087D0005C5A09F440C0B301A201C1015FD8611520
:1087E000710581059105A9F501E010E020E030E078
:1087F000B301A201C101E6D92B013C01611571054C
:108800008105910509F4C2C062507109810991097D
:10881000D10158962D913C91599740E050E00E942B
:10882000A059F101A28CB38CC48CD58CE68CF78C4A
:1088300000A111A10E94355A288B398B4A8B5B8B82
:108840006C8B7D8B8E8B9F8BB301A201C101E7DE08
:1088500094C02B013C01B301A201C10192DB2A8328
:108860003B834C835D836E837F834C01D10158969B
:108870008D919C9159978C0120E030E040E050E0D0
:10888000BA0119872A873B874C875D876E877F8768
:108890002A813B814C815D816E817F81C4015801B9
:1088A000C12CD12CE12CF12C00E010E00E94355AB3
:1088B000288F398F4A8F5B8F6C8F7D8F8E8F9F8F24
:1088C0001A81188B2B81298B3C813A8B4D814B8BE4
:1088D0005E815C8B6F816D8B8E8A9F8A1886D10139
:1088E000ED91FC910190F081E02DEE24E394F12CC8
:1088F0008E010F5F1F4F2A813B814C815D816E810C
:108900007F81C4010995882309F440C08981853E8F
:1089100011F0811118C0B885BF5FB887E8A1BE17F4
:1089200060F52A813B814C815D816E817F81C4012C
:10893000A0E20E943E5A2A833B834C835D836E8370
:108940007F834C012ACF2A813B814C815D816E81DE
:108950007F81C401A0E20E943E5A288B398B4A8B4A
:108960005B8B6C8B7D8B8E8B9F8B2A833B834C83A5
:108970005D836E837F834C010FCF288939894A89B3
:108980005B896C897D898E899F8908C020E030E0F1
:1089900040E050E060E070E080E090E0A096E2E12E
:1089A0000C94E359A9E4B0E0E8EDF4E40C94C75961
:1089B0009FA38EA3009709F422C2DC0114968D9127
:1089C0009C911597892B09F41AC216968D919C914A
:1089D0001797892B09F413C28091FC049091FD0430
:1089E000892B09F00CC242E350E060E070E08CEFAC
:1089F00094E00E948C5A0EA11FA11093FD040093D5
:108A0000FC04D80119966D917D918D919C911C97D4
:108A100020E032E040E050E00E94A059322E232EA8
:108A20006A0168AB79AB8AAB9BABABE00E943E5A64
:108A3000D801ED91FC91A5E2EA2EF12C8E010F5F99
:108A40001F4F0995811105C01092FD041092FC047E
:108A5000D6C1CE0101960E9400519FA78EA7CE01DC
:108A600004960E9400518C01BB81BEAFEE81EFAF36
:108A7000CE0107960E94005122969FAF8EAF22979B
:108A8000CE0109960E9400513C01CE010C960E9435
:108A9000005199AF88AFCE0146960E9408514B0114
:108AA0005C01CE014A960E9408516CAB7DAB8EAB47
:108AB0009FABCE0182960E9408512A966CAF7DAF83
:108AC0008EAF9FAF2A9781149104A104B10439F4A9
:108AD0006114710409F4B8CF4301A12CB12CE8ACA6
:108AE000F9ACE114F10441F0C701A0E0B0E08CABB7
:108AF0009DABAEABBFAB09C08CA99DA9AEA9BFA968
:108B0000892B8A2B8B2B09F49FCF24013501401A26
:108B1000510A610871089FAD892F90E0A0E0B0E094
:108B200026968CAF9DAFAEAFBFAF26972CA93DA9BF
:108B30004EA95FA9BC01CD010E94AA58461A570A46
:108B4000680A790A8EA59FA5019722962EAD3FADA2
:108B50002297B5E0220F331FBA95E1F7820F931FDA
:108B60006EA57FA50E94C558461A570A610871086C
:108B7000AEAD2A2F30E040E050E0C301B2010E94C8
:108B8000EC582AAF3BAF4CAF5DAF253FBFE03B0792
:108B90004105510508F458CF253F3F4F4105510588
:108BA00030F486E0AEA1BFA118968C9304C08BE090
:108BB000EEA1FFA180874CE250E060E070E08EEF14
:108BC00094E00E948C5AEEA4FFA42701612C712C22
:108BD000C501B401A30192010E94A0592093FE0493
:108BE0003093FF0440930005509301056093020504
:108BF000709303058093040590930505B80180E008
:108C000090E0A30192010E94A059A32CB22CE8A8E5
:108C1000F9A80AA91BA90E94355A28AB39AB4AAB5F
:108C20005BAB1B014C012093060530930705409375
:108C300008055093090560930A0530920B0580934F
:108C40000C0590920D056AAD7BAD8CAD9DAD6E5F50
:108C50007F4F8F4F9F4FAEA1BFA118962C9126300A
:108C600029F422E030E040E050E004C024E030E0AD
:108C700040E050E00E94AA5860930E0570930F05E3
:108C80008093100590931105EEA5FFA5F0931305B1
:108C9000E0931205AEACAE9EC001AF9E900D1124C4
:108CA0009093150580931405AEA1BFA118968C91E1
:108CB000863009F057C0E8ADF9AD9F0140E050E0C3
:108CC000C301B2010E94A059AFACB12CC12CD12C70
:108CD000E12CF12C00E010E00E944F59A8A8B9A89F
:108CE000CAA8DBA8710184010E94355A19012A0122
:108CF0003B014C0120931E0530921F054093200537
:108D000050922105609322057092230580932405DB
:108D1000909225052296AEACBFAC2297B50180E0BB
:108D200090E020E230E040E050E00E94A05959017C
:108D30006A017B018C019101A201B301C4010E946F
:108D4000355A209316053093170540931805509314
:108D5000190560931A0570931B0580931C05909369
:108D60001D054AC0CEA4DFA4B60180E090E026969F
:108D70002CAD3DAD4EAD5FAD26970E94A059CCA85D
:108D8000DDA8EEA8FFA856016701E12CF12C8701B0
:108D9000AEA2BFA2C8A6D9A6EAA6FBA60CA71DA78D
:108DA000E12CF12C00E010E00E944F59A8A8B9A8CE
:108DB000CAA8DBA8710184010E94355A20931605C8
:108DC00030931705409318055093190560931A05C1
:108DD00070931B0580931C0590931D052A96ECAC9F
:108DE000FDAC0EAD1FAD2A97E0922605F092270547
:108DF00000932805109329058CEF94E002C080E0D1
:108E000090E0C75BDF4FE2E10C94E359009719F063
:108E1000FC01118210820895EF92FF920F931F932D
:108E2000CF93DF937C018B01009799F06115710559
:108E300081F0FB0180A184FD0CC0809176049091AB
:108E40007704892B49F08091B9049091BA04892B59
:108E500031F080E090E024C0C6E7D4E002C0C9EB66
:108E6000D4E045E350E0B801CE0102960E94835A57
:108E7000F982E8821FAA18AE19AE1AAE1BAE1CAE5C
:108E80001DAE1EAE9E01215C3F4FF80185A196A14B
:108E9000A7A1B0A5F90180839183A283B383CE01FA
:108EA000CDB7DEB7E6E00C94EF59CF93DF93EC013A
:108EB000009741F0BC016E5F7F4F8881998116DA7F
:108EC00019821882DF91CF910895ACE1B0E0EBE612
:108ED000F7E40C94C7599A8F898F7E8B6D8B5A8BD0
:108EE000498BDC01D796BC91B983FC01F0ADFA83C4
:108EF000DC01D996BC91BB83FC01F2ADFC83DC01A3
:108F0000DB96BC91BD83FC01F4ADFE83DC01DD96F4
:108F1000BC91BF83FC01F6ADF887DC019B964D90B8
:108F20005D906D907C909E974A019A0140E050E0E0
:108F300060E070E080E090E0A980BA80CB80DC80C7
:108F4000ED80FE800F8118850E94355A6301520121
:108F5000E12CF12C87014986BA86CB86DC86ED862A
:108F6000FE860F87188BE12CF12C00E010E00E94A8
:108F7000535A41F038F06201E980FA80CE18DF08D8
:108F8000DA8AC98A09891A890115110509F420C1EB
:108F9000A98DBA8DED91FC911197A08CB18CBC8AF2
:108FA000AB8AFD01FF96408051806280738041143E
:108FB00051046104710409F050C097964D905D9082
:108FC0006D907C909A974114510461047104A9F446
:108FD000E1E0F0E029813A814B815C816D817E8105
:108FE0008F819885A0E00E945C5A11F4E0E0F0E0E7
:108FF000882799278E1B9F0BEDC029813A814B81D1
:109000005C816D817E818F819885A0E00E945C5A91
:1090100021F1C980DA80EB80FC800B891C89480132
:10902000A12CB12CC814D904EA04FB04B0F0C81870
:10903000D908EA08FB08B301A201A98DBA8D8D9168
:109040009C910E944E3C2B013C01611571058105EC
:10905000910541F78FEF9FEFBDC0EB89FC893197F8
:10906000A980BA80EA21FB21FA87E98729883A8812
:10907000098D1A8D015C1F4F1A830983A98DBA8D42
:109080000D911C91B301A201C8010E94C13F590179
:109090006A017B018F8B988F8B889C88E985FA8584
:1090A0008E1A9F0A2814390408F44101D8010D9042
:1090B000BC91A02DBC8FAB8FE985FA859F0140E064
:1090C00050E060E070E080E090E00F89188D0E9431
:1090D000355AAB8DBC8DED91FC9174010D891E89C3
:1090E0000995882309F460C0ED89FE89E80DF91D12
:1090F000FE8BED8B28183908940140E050E060E0C9
:1091000070E080E090E0A98DBA8DD796AC90D797AB
:10911000D896BC90D897D996CC90D997DA96DC900F
:10912000DA97DB96EC90DB97DC96FC90DC97DD968B
:109130000C91DD97DE961C91DE970E94355AD796EA
:109140002C93D797D8963C93D897D9964C93D99788
:10915000DA965C93DA97DB966C93DB97DC967C93DC
:10916000DC97DD968C93DD97DE969C93DE97E98500
:10917000FA858E0E9F1EAB88BC888A149B04D8F09B
:10918000B301A2018D919C910E944E3C2B013C01A8
:10919000611571058105910561F4A981BA811D925E
:1091A0001D921D921C92139789899A89821993099D
:1091B00011C01A861986E981FA8140825182628241
:1091C00073822114310409F059CF89899A8902C028
:1091D00080E090E06C96E2E10C94E359A4E1B0E009
:1091E000E4EFF8E40C94C7599C8B8B8B7C876B87DE
:1091F0005E874D87892B19F48FEF9FEFDCC12B859C
:109200003C85232BC9F38D859E85892BA9F3AB89DA
:10921000BC89D796BC91B983EB89FC89F0ADFA8300
:10922000AB89BC89D996BC91BB83EB89FC89F2AD33
:10923000FC83AB89BC89DB96BC91BD83EB89FC893F
:10924000F4ADFE83AB89BC89DD96BC91BF83EB890D
:10925000FC89F6ADF887EB89FC8983A594A5A5A5C3
:10926000B6A51C012D01612C712C430129813A8185
:109270004B815C816D817E818F8198855101620176
:10928000E12CF12C00E010E00E94535A11F008F09C
:10929000B3CF0190F081E02D208D318D3A87298761
:1092A000AB89BC89DF964D905D906D907C901901E3
:1092B00031E0231A310889819A8128223922411408
:1092C00051046104710409F081C0AB89BC8997968F
:1092D0004D905D906D907C909A974114510461047B
:1092E000710419F529813A818F819885A0E00E9447
:1092F0005C5A09F081CF01E010E020E030E040E06E
:1093000050E0BA01CF010E94E23D2B013C01EB8904
:10931000FC8967A370A781A792A7611571058105D4
:10932000910519F480E090E046C1AB89BC89D796DD
:109330001C91D797D896BC91EB89FC8901ADF2AC12
:1093400063AD74AD212F3B2F402F5F2D85AD96ADC2
:10935000A0E00E945C5AD1F1812E9B2EA02EBF2C42
:1093600029853A856901E12CF12C8C149D04AE0409
:10937000BF0460F18C189D08AE08BF08B301A201BC
:10938000AB89BC898D919C910E944E3C6115710501
:1093900081059105C1F481149104A104B10409F07F
:1093A0002BCF01E010E020E030E0B301A201EB8917
:1093B000FC89808191810E94E23D611571058105E2
:1093C000910509F4AFCF2B013C01CFCF2D853E8510
:1093D0003A8329838B899C89CF969A8B898BAB8919
:1093E000BC890D90BC91A02DB88BAF87B301A201B1
:1093F000CD010E94C13F59016A017B018C01898422
:109400009A8482189308E981FA81E815F90508F42D
:109410004F01AF85B889ED91FC91910140E050E09A
:1094200060E070E080E090E00E94355A0480F581B1
:10943000E02D74010B851C850995882309F489C0EA
:10944000EB85FC85E80DF91DFC87EB8729813A81C6
:10945000281939093A832983940140E050E060E0FB
:1094600070E080E090E0AB89BC89D796AC90D7974C
:10947000D896BC90D897D996CC90D997DA96DC90AC
:10948000DA97DB96EC90DB97DC96FC90DC97DD9628
:109490000C91DD97DE961C91DE970E94355AD79687
:1094A0002C93D797D8963C93D897D9964C93D99725
:1094B000DA965C93DA97DB966C93DB97DC967C9379
:1094C000DC97DD968C93DD97DE969C93DE97820C7D
:1094D000931CE985FA858E169F0678F1B301A201E7
:1094E0008D919C910E944E3C6115710581059105FD
:1094F00001F529813A81232B41F4A989BA891D926A
:109500001D921D921C92139724C001E010E020E0F0
:1095100030E0B301A201EB89FC89808191810E9436
:10952000E23D2B013C01611571058105910519F49E
:10953000E4CF2B013C01212C312CA989BA894D9211
:109540005D926D927C921397E981FA81EF2B09F07D
:1095500046CFEB89FC89B7A9A0ADF1ADF987EB89BE
:10956000FC89F2ADFB87EB89FC8963AD74AD03A583
:1095700014A525A536A518012901612C712C4301DC
:109580002B2F3A2F49855B8585AD96AD5101620140
:10959000E12CF12C00E010E00E94535A31F028F049
:1095A0009D0133A724A745A756A78D859E852981B0
:1095B0003A81821B930B6496E2E10C94E359A0E19B
:1095C000B0E0E5EEFAE40C94C7594C012A013B01E6
:1095D000009711F480E097C1DC019796CD90DD9063
:1095E000ED90FC909A97ED91FC91808D918DC11436
:1095F000D104E104F10461F04D825E826F827886CD
:109600008C0120E030E00D871E872F87388B24C027
:10961000411551056105710579F724C1B701A6010E
:10962000D4018D919C910E944E3C6115710581057C
:10963000910521F1ED80FE800F8118852D853E85F5
:109640004F855889E21AF30A040B150BED82FE824E
:109650000F8318876B017C014D815E816F81788556
:109660008D859E85AF85B88984179507A607B707AE
:10967000A8F2C114D104E104F10489F56D857E8559
:109680008F8598890D811E812F813885600F711F0C
:10969000821F931F61507109810991092D853E85B3
:1096A0004F8558890E94EC5889019A01B701A6019B
:1096B000D4018D919C910E94E23D61157105810557
:1096C000910509F487CFC114D104E104F10439F400
:1096D000F40167A370A781A792A76B017C01D40155
:1096E0009B964D925D926D927C929E97411451048F
:1096F0006104710429F4F40117A210A611A612A6A0
:10970000B4016E5F7F4FD4018D919C910E94764190
:10971000882309F45FCF411451046104710431F4CA
:10972000B701A601F401808191819AC00D811E814B
:109730002F8138854D855E856F8578894017510763
:109740006207730708F48EC0D4012D903C90211459
:10975000310409F487C0B2E0CB16D104E104F1046E
:1097600008F480C0B701A601C1010E944E3C6D8380
:109770007E838F839887D101ED91FC918085048150
:1097800015811E870D878B3071F58FEF9FEFAFEF3F
:10979000BFE089839A83AB83BC83C701B60124E011
:1097A00030E040E050E00E94A059D1011A96AC9000
:1097B0001A971B96BC901B971C96CC901C971D96D5
:1097C000DC901D971E96EC901E971F96FC901F979D
:1097D00050960C91509751961C910E94355A04E076
:1097E000E02EF12C29C08FEF9FEF9A838983C70168
:1097F000B60122E030E040E050E00E94A059D101E3
:109800001A96AC901A971B96BC901B971C96CC90FE
:109810001C971D96DC901D971E96EC901E971F9628
:10982000FC901F9750960C91509751961C910E9456
:10983000355A12E0E12EF12C8E010F5F1F4FED859E
:10984000FE850995882371F0ED80FE800F811885D3
:10985000E114F1040105110529F0B801A701C101C6
:109860000E94DB3C9301820140E050E0BA014D824E
:109870001E832F83388749875A876B877C87D4015B
:10988000D796AC90D797D896BC90D897D996CC90CD
:10989000D997DA96DC90DA97DB96EC90DB97DC963A
:1098A000FC90DC97DD960C91DD97DE961C91DE979F
:1098B0002D813E814F81588560E070E080E090E02E
:1098C0000E94535AF8F4D7962C93D797D8963C9386
:1098D000D897E42ED9964C93D997F52EDA965C93C7
:1098E000DA97DB961C92DB97DC961C92DC97DD9670
:1098F0001C92DD97DE961C92F401FF961082118275
:109900001282138281E06096E2E10C94E359A0E0B8
:10991000B0E0EDE8FCE40C94C959EC018B01009730
:1099200009F453C06115710509F44FC06FA958AD12
:1099300039AD2AAD4130A1F068F0423009F045C0A0
:10994000F80140805180628073808BA59CA5ADA5F5
:10995000BEA50FC0F80140805180628073800DC0A9
:10996000862F952FA32FB22FF8014080518062805F
:109970007380480E591E6A1E7B1E8BA59CA5ADA543
:10998000BEA584159505A605B705C8F0530142018B
:10999000C12CD12C76014FAA98AEA9AEBAAE1BAE9F
:1099A0001CAE1DAE1EAEEF96188219821A821B8263
:1099B000F801408251826282738281E007C0B30164
:1099C000A201CE01FCDD8111E1CF80E0CDB7DEB791
:1099D000E0E10C94E559EF92FF920F931F93CF9320
:1099E000DF937C018B01009791F06115710579F08F
:1099F000FB0180A184FF0BC0C5E4D3E0888199817D
:109A0000892B41F0ED96F4E0C637DF07B9F780E027
:109A100090E015C045E350E0B801CE0102960E94E7
:109A2000835AF982E882F80185A196A1A7A1B0A581
:109A30008FAB98AFA9AFBAAF1CAE1BAECE01CDB7FE
:109A4000DEB7E6E00C94EF59009719F0FC011182A3
:109A500010820895FC01009761F047A150A561A50F
:109A600072A547AB50AF61AF72AF14AE13AE81E0D9
:109A7000089580E00895A6E3B0E0E1E4FDE40C94ED
:109A8000C7599AA789A78B01892B01F16115710527
:109A9000E9F0A9A5BAA52D903C901197F101008C91
:109AA000F18DE02DFCA7EBA7D7964D905D906D90C2
:109AB0007C90DA97DB962D913C91DC9738A72FA309
:109AC0002E173F0728F089A59AA5C4DF80E0CCC0F7
:109AD00046E050E060E070E0CE0181960E948C5A32
:109AE00045E350E060E070E0C8010E948C5A1AA380
:109AF00009A3411451046104710409F080C0D1012B
:109B0000ED91FC91119780858B3039F49A964D90A8
:109B10005D906D907C909D9772C0F101028CF38DE9
:109B2000E02DD10192968D919C919397E81BF90BB2
:109B3000FCA7EBA764C0EBA5FCA52FA138A5E21BF1
:109B4000F30BFEABEDABA90160E070E080E090E0CC
:109B5000DC012DA75EA76FA778AB89AB9AABABAB47
:109B6000BCAB411451046104710409F04DC040E0E4
:109B700050E060E070E080E090E0D1019296AC901F
:109B800092979396BC9093979496CC909497959631
:109B9000DC9095979696EC9096979796FC90979771
:109BA00098960C91989799961C910E94355A1CA2F0
:109BB0001BA2D101ED91FC910280F381E02DDE0129
:109BC00091964D01AAE2AA2EA0E4BA2ECDA8DEA855
:109BD000B0E2EB2EF12C8E010F5F1F4F0995882309
:109BE00009F474CF8BA19CA1EFA1F8A5E80FF91F90
:109BF000F8A7EFA32BA53CA5E217F30798F48EA1D5
:109C0000882309F498CF21C0B301A201C1010E94A9
:109C1000C13FADA4BEA4C12CD12CE12CF12C00E09D
:109C200010E0C3CFB301A201C1010E944E3C2B0141
:109C30003C01611571058105910521F48EA1811109
:109C400004C041CF18A61FA2DACFA9A5BAA5D796FE
:109C50004D925D926D927C92DA97EFA1F8A5DC9619
:109C6000FC93EE93DB978EA1E696E2E10C94E35928
:109C7000A0E0B0E0EEE3FEE40C94CD595C01EB0112
:109C80008A01009709F45EC0209709F45BC08881BF
:109C9000882309F457C04115510509F453C08F3288
:109CA00009F4219645E350E060E070E0C8010E94AD
:109CB0008C5A80E1F80180A38881811102C081E083
:109CC00042C0B801C50187DE7C010097D9F16FE27F
:109CD00070E0CE010E949E5A009741F0C82ECC1A27
:109CE0004C012FEF821A920AD12C0EC0CE010E9495
:109CF000CD5AC82E4E01880E911CF6CFC8010E9485
:109D0000CD5A8C159D0531F0B801C701B4DE811123
:109D1000F5CF15C0A601B801CE010E94D65A892BF5
:109D200099F7C70191DECC0DDD1D8881882339F2BA
:109D3000F80180A184FF06C0E401E12CF12CC701E9
:109D400083DEBACF80E0CDB7DEB7ECE00C94E95902
:109D5000A0E0B0E0EEEAFEE40C94D1598C017B0166
:109D6000EA01009709F443C06115710509F43FC089
:109D7000FB0180818823D9F12097C9F1BE01C80178
:109D80007ADE882351F0BE01C7010E94A95A892BAF
:109D9000A9F7C8015FDE92E02BC0F801C080D18036
:109DA00045E350E060E070E0CE010E948C5A4FE144
:109DB00050E0B701CE010E94E45AB801695D7F4FBF
:109DC000AE01C6010E9449432DA73EA74FA758AB3D
:109DD00069AB7AAB8BAB9CABA0E00E945C5A39F0CC
:109DE000BE01C6010E94764191E0811101C090E060
:109DF000892FCDB7DEB7E8E00C94ED59FC01009750
:109E000011F1A081B18118964C9182899389A4891E
:109E1000B589208D318DBC01CD014B3041F4F2E08C
:109E20009695879577956795FA95D1F704C096959D
:109E3000879577956795625071098109910940E08E
:109E400050E00C94A05920E030E040E050E060E0A9
:109E500070E080E090E00895A0E3B0E0E2E3FFE48A
:109E60000C94C7593C01009749F420E030E040E0F1
:109E700050E060E070E080E090E091C019A21AA28A
:109E80001BA21CA280E290E09EA38DA3F301F285A9
:109E9000F9A7F301F385FAA7F301F485FBA7F30112
:109EA000F585FCA7F301F685FDA7F301F785FEA76D
:109EB000F301F089FFA7F301F189F8ABF3012288E0
:109EC000338844885588211431044104510409F42D
:109ED0005BC0FEEF2F16FFEF3F064104510418F45C
:109EE00038A62FA204C02EEF3FEF38A72FA3A895C6
:109EF000F301A081B1811296ED91FC911397189610
:109F00008C91863019F48FEF9FE302C089E491E4CD
:109F10009E012F5D3F4F49015C01CFA0D8A4A0E274
:109F2000EA2EF12C8E010F5F1F4F29A53AA54BA5F4
:109F30005CA56DA57EA58FA598A90995882309F430
:109F400094CFCFA0D8A44601960140E050E060E055
:109F500070E080E090E0A9A4BAA4CBA4DCA4EDA4B6
:109F6000FEA40FA518A90E94355A29A73AA74BA706
:109F70005CA76DA77EA78FA798AB8FA198A5281A7D
:109F8000390A410851089FCF69A17AA18BA19CA1F0
:109F9000F301208D318D40E050E00E94A059E09601
:109FA000E2E10C94E359AEE0B0E0E9EDFFE40C949B
:109FB000C7591B011E861D869C0140E050E0298781
:109FC0003A874B875C8700E911E08D859E85821575
:109FD000930509F406C1809107018093840060E233
:109FE00071EA87E090E029853A854B855C850E947F
:109FF0000E59CA01B90197D74B015C012BEA3AEA25
:10A000004AEA50E40E9447586B017C0120E030E0AE
:10A0100040E850E4C501B4010E9447582B013C01BF
:10A0200020E030E040E85FE3C701B601E2D687FDFB
:10A0300066C020E03FEF4FE757E4C301B2010E9442
:10A04000435818160CF047C020E030E04AE754E4CB
:10A05000C501B401D2D66D837E838F83988720E0BB
:10A0600030E04AE755E40E94475869837A838B833E
:10A070009C8320E030E040E85FE3BBD687FD24C04E
:10A0800020E03FEF4FE757E469817A818B819C8123
:10A09000FAD718169CF420E030E040E251E46D81DC
:10A0A0007E818F819885F3D710D76115710589F06E
:10A0B000C8010197F1F761507109F7CF69817A8181
:10A0C0008B819C8102D702C061E070E0CB010197D7
:10A0D000F1F760E015C020E030E04FE753E4C7013E
:10A0E000B601D1D718163CF4C301B201EED6CB01AC
:10A0F0000197F1F707C0C701B601E7D601C061E0DB
:10A100006A95F1F71092840020E030E040E85FE3C8
:10A11000C701B6016ED687FD5AC020E03FEF4FE77A
:10A1200057E4C301B201AFD718160CF03CC020E0D1
:10A1300030E04AE754E4C501B4015FD64B015C014D
:10A1400020E030E04AE755E4A2D76B017C0120E033
:10A1500030E040E85FE34DD687FD1EC020E03FEFD2
:10A160004FE757E4C701B6018ED718168CF420E0EC
:10A1700030E040E251E4C501B40189D7A6D66115AB
:10A18000710579F0C8010197F1F761507109F7CFB6
:10A19000C701B6019AD602C061E070E0CB01019719
:10A1A000F1F760E015C020E030E04FE753E4C7016D
:10A1B000B60169D718163CF4C301B20186D6CB01AB
:10A1C0000197F1F707C0C701B6017FD601C061E072
:10A1D0006A95F1F74D855E854F5F5F4F5E874D87CE
:10A1E000F4CE2E96E2E10C94E359EBE8F0E08081A6
:10A1F00081628083EAE8F0E080818960808308954D
:10A20000FC01818190E0982F88272081822B08957E
:10A21000FC0123816281862F90E0A0E0B0E07727E7
:10A220006627922B2081622B2181722B0895FC01DD
:10A23000718360830895FC0173836283518340833B
:10A24000089541E050E063EF77E08091330590910D
:10A2500034050E9465478091F3070895A5E3B0E0B7
:10A26000E4E3F1E50C94D1597C018B016A01CB0147
:10A27000F1DBBE016F5F7F4FC801FDDB882381F0FA
:10A28000B601CE0101960E94A95A892B91F7C80107
:10A29000E1DBBE016F5F7F4FC7010E940C4704C026
:10A2A000C801D8DB80E090E0E596E8E00C94ED5939
:10A2B00080913105882351F18091F60980FF11C00A
:10A2C00040E052E063EF77E08091330590913405F0
:10A2D0000E94EE480E94BF0D8091F6098E7F809308
:10A2E000F6098091F60981FF11C040E052E064E573
:10A2F0007CE080913305909134050E94EE480E94E5
:10A30000BF0D8091F6098D7F8093F609089587EF40
:10A3100099E0089589EC97E00895BC0183ED97E0FA
:10A320000C94B25A0895BC0183ED97E00C94735AD3
:10A33000089583ED97E00895CF93DF93EC0183EDCB
:10A3400097E00E94CD5AFC01FF27ED52F84FDF0144
:10A3500011978FE28C931082BE0183ED97E00E94EB
:10A36000935ADF91CF91089583ED97E00E94CD5AE3
:10A37000813081F0815020E030E0E82FE21BF0E0F6
:10A380002F5F3F4FED52F84F90819F32B1F711820E
:10A3900081E0089580E0089580913B05882349F18C
:10A3A0008091350590913605009729F04DDB10928C
:10A3B0003605109235058091370590913805009744
:10A3C00031F00E94064710923805109237058091AF
:10A3D000390590913A05009731F00E94670C109270
:10A3E0003A05109239051092C8071092C7071092CB
:10A3F0003B050895E0913305F091340563A574A5FC
:10A4000085A596A50895CF93DF936091350570914A
:10A410003605AC0180913705909138051FDFEC01BE
:10A4200090933405809333050E94554781E0CD2BEE
:10A4300009F480E0DF91CF910895E091F309F09164
:10A44000F4090995089580913205882309F442C0E2
:10A450008091C60781113EC08091F60980FD12C02F
:10A4600040E052E063EF77E080913305909134054E
:10A470000E9465472091F60921602093F609811515
:10A480009240B0F08091F60981FD24C040E052E096
:10A4900064E57CE080913305909134050E94654726
:10A4A0002091F60922602093F6098115924090F4DC
:10A4B00081E08093C6078091C7079091C807892BD8
:10A4C00049F0E091C707F091C80709951092C807B5
:10A4D0001092C7070895E091520CF091530C099522
:10A4E00008950E94BF0DE4DE80913105882309F4B0
:10A4F0004BC08091520C9091530C8555974021F49C
:10A500004091F50950E016C08091520C9091530C87
:10A510008856974021F44091F50950E019C0809188
:10A52000520C9091530C8B57974039F44091F50998
:10A5300050E0539563EF77E00DC08091520C9091FD
:10A54000530C8359974071F44091F50950E05395AD
:10A5500064E57CE080913305909134050E94EE48DB
:10A560008091F5090E94BF0D1092F6091092F5092D
:10A5700085E197E09093F4098093F3098BEA97E0E3
:10A580009093530C8093520C0895ABDF8091330568
:10A5900090913405009731F00E9455471092340590
:10A5A000109233051092320510923105089599DF0B
:10A5B0008091330590913405FC0147A950AD61AD00
:10A5C00072AD0E94DF4AE0913305F091340567A92E
:10A5D00070AD81AD92AD0895E0913305F0913405F1
:10A5E00047A950AD61AD72ADFC01408351836283D8
:10A5F00073830895A4E0B0E0EFEFF2E5D8C6698375
:10A600007A838B839C8340E0BE016F5F7F4F809194
:10A610003305909134057BD991E0811101C090E020
:10A620002091F3093091F4092152314561F01092E3
:10A63000F60925E137E03093F4092093F3091092ED
:10A64000F5091092C607892F2496E2E0CCC6A4E053
:10A65000B0E0ECE2F3E5ABC69B01AC01882799279B
:10A66000DC01821B930BA40BB50B89839A83AB830C
:10A67000BC8342E0BE016F5F7F4F809133059091B4
:10A68000340545D991E0811101C090E02091F30992
:10A690003091F4092152314561F01092F60925E11B
:10A6A00037E03093F4092093F3091092F5091092E2
:10A6B000C607892F2496E2E096C6C5DEF9CD089537
:10A6C000CF92DF92EF92FF92CF93DF93CDB7DEB7B9
:10A6D000E5970FB6F894DEBF0FBECDBFC12CD12CCD
:10A6E0007601BE016F5F7F4F8091350590913605F1
:10A6F000C2D9882349F089818E3299F38FEFC81A25
:10A70000D80AE80AF80AEDCF809135059091360510
:10A71000A1D9C701B601E5960FB6F894DEBF0FBE0A
:10A72000CDBFDF91CF91FF90EF90DF90CF90089554
:10A730000F930E94290F91E0811101C090E0909346
:10A740003B05992309F468C000E02FE531E14DE5B0
:10A7500050E16DEE7FE08BEE9DE00E94EE0B90935A
:10A760003A0580933905892B79F40FEF2FE531E114
:10A770004DE550E16DEE7FE08BEE9DE00E94EE0B2B
:10A7800090933A05809339058091390590913A0567
:10A79000009709F441C00E94D244909338058093F9
:10A7A00037050097C9F14DE15CE063ED77E060DAD1
:10A7B00081110EC08FE28093D3071092D4074DE130
:10A7C0005CE063ED77E0809137059091380550DAD1
:10A7D0006DE17CE08091370590913805FCD890932D
:10A7E000360580933505892BB9F06ADF6093CB0776
:10A7F0007093CC078093CD079093CE071092CF072C
:10A800001092D0071092D1071092D2071092CA0767
:10A810001092C90781E001C080E00F910895CF93A5
:10A82000DF93EC0180913B05811101C081DF6091D4
:10A83000350570913605AE01809137059091380548
:10A840000DDD9093340580933305892BD1F0109260
:10A85000F6091092C60785E197E09093F40980937A
:10A86000F3091092F50981E08093320510923105C9
:10A87000109233011092C8071092C707E4DD81E0FF
:10A8800001C080E0DF91CF910895A9E3B0E0EAE450
:10A89000F4E58BC58C01AE014F5F5F4FBC01809129
:10A8A00035059091360554DA811102C010E027C0B9
:10A8B0000E94BF0DC801B3DF182F8823B9F31EAA69
:10A8C0001FAA18AE19AE40E0BE016A5C7F4F8091AE
:10A8D0003305909134051BD8882341F30E94BF0DA6
:10A8E0001092F6092BEA37E03093530C2093520C68
:10A8F0001092F5091092320581E080933105812F85
:10A90000E996E4E06EC5A5E3B0E0E8E8F4E545C506
:10A910006B017C0180913B05811101C009DF8091B1
:10A92000CF079091D007A091D107B091D207C81658
:10A93000D906EA06FB0639F4C114D104E104F10496
:10A9400009F0F9C00AC0C816D906EA06FB0628F0C5
:10A95000C114D104E104F10439F5809135059091D9
:10A96000360578D8812C912C54018C149D04AE04AA
:10A97000BF0408F050C0BE016F5F7F4F8091350566
:10A980009091360578D8882309F440C089818E32A9
:10A9900029F421E0821A9108A108B1086FEF861A04
:10A9A000960AA60AB60AE1CF8C159D05AE05BF052D
:10A9B000B0F52091C9073091CA074C015D01820EA4
:10A9C000931EA11CB11CC814D904EA04FB0408F4AA
:10A9D0006DC00DC089818E3229F421E0821A910860
:10A9E000A108B1086FEF861A960AA60AB60A8C1457
:10A9F0009D04AE04BF0478F4BE016F5F7F4F809169
:10AA000035059091360537D88111E4CF1092CA07E9
:10AA10001092C90790C01092CA071092C90700E0AF
:10AA200010E0C092CF07D092D007E092D107F09209
:10AA3000D2078EE3F82EBE016F5F7F4F8091350500
:10AA40009091360518D8882309F475C089818E3213
:10AA500091F3CE010196A1D5E82E89A184FF06C00D
:10AA6000F801E950F64FF0820F5F1F4FBE016F5F94
:10AA70007F4FC8018950964F75D5C8018E0D911D25
:10AA80008C010F5F1F4FFC01E950F64F108220919F
:10AA9000C9073091CA072F5F3F4F3093CA072093F1
:10AAA000C90783968532924030F245C04C015D0162
:10AAB00040E050E04F5F5F4FFA01EA50F64F60818F
:10AAC0006111F8CF6FEF861A960AA60AB60A8C149F
:10AAD0009D04AE04BF0471F746015701881A990A14
:10AAE000AA0ABB0A2819390980E090E000E010E0CA
:10AAF00082179307D9F0401B510BDA01A950B64FCA
:10AB0000BA01600F711FFD01E00FF11FB080F80165
:10AB1000E950F64F0F5F1F4FBB2011F0B082F0CF0E
:10AB2000AB014F5F5F4F10820196E2CF9093CA074F
:10AB30008093C90776CFE596ECE04BC4A5E3B0E07F
:10AB4000E3EAF5E52CC45C0180913505909136056A
:10AB50000E942A4DC12CD12C7601BE016F5F7F4F20
:10AB600080913505909136050E943B4D0091350549
:10AB700010913605811114C0C8010E942A4D10920F
:10AB8000CF071092D0071092D1071092D2071092DF
:10AB9000CA071092C9076FEF7FEF8FEF9FEF22C0B8
:10ABA00089818E32D1F2BE016F5F7F4FC501D1D452
:10ABB000892B91F4C8010E942A4D1092CF07109260
:10ABC000D0071092D1071092D2071092CA071092A4
:10ABD000C907B601C70106C08FEFC81AD80AE80A2C
:10ABE000F80ABBCFE596EAE0F6C380913305909171
:10ABF000340502960895A8E0B0E0E0E0F6E5D5C39C
:10AC000080913B058111C8DB93DD882309F451C095
:10AC100083EF97E00E94DE1111E0811101C010E086
:10AC20008091370590913805E9D804E102D42D834D
:10AC30003E834F83588780913705909138050CD912
:10AC4000F8D329833A834B835C8344E050E0BE0110
:10AC50006B5F7F4F84E59CE056D444E050E0BE013A
:10AC60006F5F7F4F88E59CE04ED46091370570910F
:10AC70003805685E7F4F42E050E08CE59CE043D4AD
:10AC800060913705709138056A5E7F4F42E050E071
:10AC90008EE59CE038D4E0913705F091380560816D
:10ACA0007181685F7F4F41E050E080E69CE02BD4EB
:10ACB00001C010E071DB812F2896E4E092C383EF9E
:10ACC00097E00895A4E0B0E0E7E6F6E570C344E05D
:10ACD00050E068E57CE0CE01019615D469817A8167
:10ACE0008B819C812496E2E07EC3A4E0B0E0EAE799
:10ACF000F6E55DC344E050E064E57CE0CE010196FA
:10AD000002D469817A818B819C812496E2E06BC3B5
:10AD10009ADB93CB08951092300510922F05109274
:10AD20002E05089580913005089580912E0590910B
:10AD30002F05089581E080933301089581E02091EB
:10AD4000330530913405232B09F480E008951092E7
:10AD5000F6098BEA97E09093530C8093520C109273
:10AD6000F5091092320581E0809331050895109223
:10AD7000F60985E197E09093F4098093F309109226
:10AD8000F50981E080933205109231050895A2E023
:10AD9000B0E0ECECF6E50BC342E050E06CE57CE0A3
:10ADA000CE010196B0D389819A812296E2E01BC33D
:10ADB000A2E0B0E0EDEDF6E5FAC242E050E06EE56B
:10ADC0007CE0CE0101969FD389819A812296E2E0B0
:10ADD0000AC3A1E0B0E0EEEEF6E5E9C241E050E0E2
:10ADE00060E67CE0CE0101968ED389812196E2E077
:10ADF000FAC2D4D008F481E008950CD00AC102D17F
:10AE000040F0F9D030F021F45F3F19F0EBC0511160
:10AE100034C1EEC00FD198F39923C9F35523B1F390
:10AE2000951B550BBB27AA2762177307840738F0B9
:10AE30009F5F5F4F220F331F441FAA1FA9F333D018
:10AE40000E2E3AF0E0E830D091505040E695001CCC
:10AE5000CAF729D0FE2F27D0660F771F881FBB1F88
:10AE6000261737074807AB07B0E809F0BB0B802D62
:10AE7000BF01FF2793585F4F2AF09E3F510568F0AE
:10AE8000B1C0FBC05F3FECF3983EDCF3869577954D
:10AE90006795B795F7959F5FC9F7880F911D9695B0
:10AEA000879597F90895E1E0660F771F881FBB1F0C
:10AEB000621773078407BA0720F0621B730B840BB9
:10AEC000BA0BEE1F88F7E0950895BCD088F09F5725
:10AED00090F0B92F9927B751A0F0D1F0660F771FE6
:10AEE000881F991F1AF0BA95C9F712C0B13081F0C6
:10AEF000C3D0B1E00895C0C0672F782F8827B85F0E
:10AF000039F0B93FCCF3869577956795B395D9F726
:10AF10003EF490958095709561957F4F8F4F9F4F30
:10AF20000895E89409C097FB3EF49095809570953C
:10AF300061957F4F8F4F9F4F9923A9F0F92F96E985
:10AF4000BB279395F695879577956795B795F111FA
:10AF5000F8CFFAF4BB0F11F460FF1BC06F5F7F4F97
:10AF60008F4F9F4F16C0882311F096E911C07723A9
:10AF700021F09EE8872F762F05C0662371F096E8B2
:10AF8000862F70E060E02AF09A95660F771F881F81
:10AF9000DAF7880F9695879597F90895990F000825
:10AFA000550FAA0BE0E8FEEF16161706E807F9079B
:10AFB000C0F012161306E407F50798F0621B730B36
:10AFC000840B950B39F40A2661F0232B242B252BB7
:10AFD00021F408950A2609F4A140A6958FEF811D5A
:10AFE000811D089597F99F6780E870E060E00895FB
:10AFF0009FEF80EC089500240A9416161706180691
:10B000000906089500240A9412161306140605066C
:10B010000895092E0394000C11F4882352F0BB0FFD
:10B0200040F4BF2B11F460FF04C06F5F7F4F8F4F60
:10B030009F4F089557FD9058440F551F59F05F3F9B
:10B0400071F04795880F97FB991F61F09F3F79F04A
:10B0500087950895121613061406551FF2CF4695CC
:10B06000F1DF08C0161617061806991FF1CF86954E
:10B070007105610508940895E894BB276627772732
:10B08000CB0197F908958ADF08F48FEF08950BD06C
:10B09000C0CFB1DF28F0B6DF18F0952309F0A2CFBA
:10B0A000A7CF1124EACFC6DFA0F3959FD1F3950F68
:10B0B00050E0551F629FF001729FBB27F00DB11D3C
:10B0C000639FAA27F00DB11DAA1F649F6627B00DCC
:10B0D000A11D661F829F2227B00DA11D621F739FB5
:10B0E000B00DA11D621F839FA00D611D221F749FC3
:10B0F0003327A00D611D231F849F600D211D822F0A
:10B10000762F6A2F11249F5750408AF0E1F0882350
:10B110004AF0EE0FFF1FBB1F661F771F881F91505D
:10B120005040A9F79E3F510570F05CCFA6CF5F3F1E
:10B13000ECF3983EDCF3869577956795B795F79590
:10B14000E7959F5FC1F7FE2B880F911D9695879518
:10B1500097F90895DB018F939F9391D0BF91AF91A1
:10B16000A29F800D911DA39F900DB29F900D112461
:10B170000895991B79E004C0991F961708F0961B53
:10B18000881F7A95C9F780950895AA1BBB1B51E1CA
:10B1900007C0AA1FBB1FA617B70710F0A61BB70B47
:10B1A000881F991F5A95A9F780959095BC01CD01EC
:10B1B000089597FB072E16F4009406D077FD08D06B
:10B1C000E4DF07FC05D03EF4909581959F4F0895EC
:10B1D000709561957F4F0895A1E21A2EAA1BBB1BA3
:10B1E000FD010DC0AA1FBB1FEE1FFF1FA217B30753
:10B1F000E407F50720F0A21BB30BE40BF50B661F69
:10B20000771F881F991F1A9469F76095709580952C
:10B2100090959B01AC01BD01CF010895052E97FBD0
:10B2200016F400940FD057FD05D0D6DF07FC02D0EE
:10B2300046F408C050954095309521953F4F4F4FAB
:10B240005F4F089590958095709561957F4F8F4FD2
:10B250009F4F0895EE0FFF1F0590F491E02D099484
:10B26000A29FB001B39FC001A39F700D811D112447
:10B27000911DB29F700D811D1124911D0895F0DF65
:10B28000A59F900DB49F900DA49F800D911D11243A
:10B290000895B7FFF4CFF3DF821B930B0895DF937C
:10B2A000CF931F930F939A9DF02D219FF00D8B9DAF
:10B2B000F00D8A9DE02DF10D039FF00D029FE00D32
:10B2C000F11D4E9DE00DF11D5E9DF00D4F9DF00DA9
:10B2D0007F936F93BF92AF925F934F93D501C0DF7F
:10B2E0008B01AC01D701BCDFEB01E80FF91FD601E0
:10B2F0001FD02F913F91D601B3DFC60FD71FE81F94
:10B30000F91FAF91BF9114D02F913F91A9DFC60FC4
:10B31000D71FE81FF91FD601A3DFE60FF71F98011B
:10B32000BE01CF0111240F911F91CF91DF9108959C
:10B3300097DF460F571FC81FD91F08F4319608958D
:10B34000E894DF93CF93FC01DB018ADF7F936F9357
:10B35000E9019A01AC01BF93AF933F932F93DF01B3
:10B360007FDF26F46C1B7D0B820B930B9E01EB01A0
:10B37000FC01DEDFAF91BF912F913F91D9DFBE017C
:10B38000CF01F9012F913F91CF91DF9108952F9235
:10B390003F924F925F926F927F928F929F92AF9265
:10B3A000BF92CF92DF92EF92FF920F931F93CF93B2
:10B3B000DF93CDB7DEB7CA1BDB0B0FB6F894DEBF49
:10B3C0000FBECDBF09942A88398848885F846E846F
:10B3D0007D848C849B84AA84B984C884DF80EE80B9
:10B3E000FD800C811B81AA81B981CE0FD11D0FB6C2
:10B3F000F894DEBF0FBECDBFED0108950F93083066
:10B4000090F0982F872F762F652F542F432F322FB0
:10B4100022270850F4CF220F331F441F551F661FE9
:10B42000771F881F991F0A95B2F70F91089597FB10
:10B4300010F8169400080F93083098F00850232F46
:10B44000342F452F562F672F782F892F902DF4CF2B
:10B45000059497958795779567955795479537956F
:10B4600027950A95AAF70F9108952A0D3B1D4C1DAB
:10B470005D1D6E1D7F1D801F911F08950024A7FD77
:10B4800000942A0F301D401D501D601D701D801D31
:10B49000901D08952A193B094C095D096E097F0921
:10B4A000800B910B08952A153B054C055D056E0533
:10B4B0007F058007910708950024A7FD00942A17AF
:10B4C000300540055005600570058005900508951C
:10B4D000FB01DC010D900020E9F7119705900D921A
:10B4E0000020E1F70895FB01DC0105900D9200209A
:10B4F000E1F70895FC0105900020E9F7809590950B
:10B500008E0F9F1F0895FB01DC0102C001900D9278
:10B5100041505040D8F70895DC0101C06D9341506F
:10B520005040E0F70895FB01DC010D900020E9F7A1
:10B53000119701900D920020E1F70895FC0181918F
:10B54000861721F08823D9F7992708953197CF01DD
:10B550000895FB01DC018D91019080190110D9F350
:10B56000990B0895FB01DC0101900D920020E1F799
:10B570000895DC01FB014150504058F049F0019022
:10B580000D920020C1F7E61BF70B3197CF0108950C
:10B590001C9201900020E9F7F6CFFC0101900020F9
:10B5A000E9F7809590958E0F9F1F0895FB01DC01B0
:10B5B0004150504030F08D910190801919F40020D5
:10B5C000B9F7881B990B0895FB01DC0141505040ED
:10B5D00048F001900D920020C9F701C01D92415022
:10B5E0005040E0F70895FC0181E090E001900616DC
:10B5F00009F4CF010020D1F701970895BB274A3005
:10B6000031F4992322F4BDE2909581959F4F30C08B
:10B61000BB272A3051F4992342F4BDE290958095DE
:10B62000709561957F4F8F4F9F4F01C0BB27FA01E7
:10B63000A62F6217710581059105330B30FB66F06B
:10B64000AA27660F771F881F991FAA1FA21710F03D
:10B65000A21B63953850A9F7A05DAA3308F0A95D35
:10B66000A19336F7B111B1931082CA018CC2BB27E6
:10B67000FB015527AA27880F991FAA1FA41710F0AE
:10B68000A41B83955051B9F7A05DAA3308F0A95DBA
:10B69000A193009779F7B111B1931192CB0173C2C5
:10B6A0000F931F93CF93DF93CDB7DEB72E970FB6CF
:10B6B000F894DEBF0FBECDBF0D891E898EE08C834E
:10B6C0001A8309838FEF9FE79E838D83AE01475EC8
:10B6D0005F4F6F89788DCE01019610D0EF81F8858C
:10B6E000E00FF11F10822E960FB6F894DEBF0FBE4A
:10B6F000CDBFDF91CF911F910F9108952F923F926F
:10B700004F925F926F927F928F929F92AF92BF9271
:10B71000CF92DF92EF92FF920F931F93CF93DF931D
:10B72000CDB7DEB72C970FB6F894DEBF0FBECDBFF6
:10B730007C016B018A01FC0117821682838181FFE3
:10B74000B0C1CE0101964C01F7019381F60193FD42
:10B75000859193FF81916F01882309F49EC1853201
:10B7600039F493FD859193FF81916F01853221F426
:10B77000B70190E018D2E8CF512C312C20E02032D4
:10B78000A0F48B3269F030F4803259F0833269F4DE
:10B7900020612CC08D3239F0803339F4216026C00D
:10B7A0002260246023C0286021C027FD27C030ED1F
:10B7B000380F3A3078F426FF06C0FAE05F9E300D6D
:10B7C0001124532E13C08AE0389E300D1124332EDD
:10B7D00020620CC08E3221F426FD5FC1206406C0B9
:10B7E0008C3611F4206802C0883641F4F60193FDCE
:10B7F000859193FF81916F018111C1CF982F9F7D1A
:10B800009554933028F40C5F1F4FFFE3F9830DC06C
:10B81000833631F0833771F0833509F057C021C08A
:10B82000F801808189830E5F1F4F44244394512C7B
:10B83000540114C03801F2E06F0E711CF801A080B1
:10B84000B18026FF03C0652D70E002C06FEF7FEF6F
:10B85000C5012C878DD12C0183012C852F77222EB9
:10B8600016C03801F2E06F0E711CF801A080B180A3
:10B8700026FF03C0652D70E002C06FEF7FEFC501AA
:10B880002C876BD12C012C852068222E830123FC70
:10B8900019C0832D90E048165906A0F4B70180E244
:10B8A00090E081D13A94F5CFF50127FC859127FEF0
:10B8B00081915F01B70190E076D131103A94F1E0C7
:10B8C0004F1A51084114510479F7DEC0843611F043
:10B8D000893631F5F80127FF07C0608171818281C7
:10B8E00093810C5F1F4F08C060817181882777FDAD
:10B8F0008095982F0E5F1F4F2F76B22E97FF09C0AD
:10B9000090958095709561957F4F8F4F9F4F2068E0
:10B91000B22E2AE030E0A40178D1A82EA81843C0A6
:10B92000853729F42F7EB22E2AE030E025C0F22F91
:10B93000F97FBF2E8F36C1F018F4883579F0ADC08D
:10B94000803719F0883721F0A8C02F2F2061B22E40
:10B95000B4FE0DC08B2D8460B82E09C024FF0AC030
:10B960009F2F9660B92E06C028E030E005C020E188
:10B9700030E002C020E132E0F801B7FE07C060818C
:10B980007181828193810C5F1F4F06C0608171813C
:10B9900080E090E00E5F1F4FA40137D1A82EA818B9
:10B9A000FB2DFF77BF2EB6FE0BC02B2D2E7FA514CF
:10B9B00050F4B4FE0AC0B2FC08C02B2D2E7E05C088
:10B9C0007A2C2B2D03C07A2C01C0752C24FF0DC0BE
:10B9D000FE01EA0DF11D8081803311F4297E09C03A
:10B9E00022FF06C07394739404C0822F867809F0F6
:10B9F000739423FD12C020FF06C05A2C731418F450
:10BA0000530C5718732C731460F4B70180E290E064
:10BA10002C87C9D073942C85F6CF731410F4371883
:10BA200001C0312C24FF11C0B70180E390E02C87C6
:10BA3000BAD02C8522FF16C021FF03C088E590E014
:10BA400002C088E790E0B7010CC0822F867851F0E1
:10BA500021FD02C080E201C08BE227FD8DE2B7012B
:10BA600090E0A1D0A51430F4B70180E390E09BD022
:10BA70005A94F8CFAA94F401EA0DF11D8081B70120
:10BA800090E091D0A110F6CF332009F45DCEB7013C
:10BA900080E290E088D03A94F7CFF70186819781D1
:10BAA00002C08FEF9FEF2C960FB6F894DEBF0FBE4B
:10BAB000CDBFDF91CF911F910F91FF90EF90DF905D
:10BAC000CF90BF90AF909F908F907F906F905F903E
:10BAD0004F903F902F900895DC01CB01FC01E1993C
:10BAE000FECF06C0FFBBEEBBE09A31960DB20D92C1
:10BAF00041505040B8F70895E199FECF9FBB8EBBEF
:10BB0000E09A99278DB30895A8E1B0E042E050E0B3
:10BB1000E5CFDC01A40FB51F4150504040F0CB01F0
:10BB2000840F951F2E9105D041505040D8F70895AD
:10BB3000262FE199FECF9FBB8EBBE09A01970DB2F5
:10BB4000021631F02DBB0FB6F894E29AE19A0FBEBF
:10BB500008950196272FEDDFEBCFFC010590615092
:10BB600070400110D8F7809590958E0F9F1F089513
:10BB7000FC016150704001900110D8F780959095BC
:10BB80008E0F9F1F0895DC01FC01672F71917723B1
:10BB9000E1F7329704C07C916D9370836291AE1788
:10BBA000BF07C8F308950F931F93CF93DF93182F08
:10BBB000092FEB018B8181FD03C08FEF9FEF20C028
:10BBC00082FF10C04E815F812C813D814217530757
:10BBD0007CF4E881F9819F012F5F3F4F39832883EF
:10BBE000108306C0E885F985812F0995892B29F7EF
:10BBF0002E813F812F5F3F4F3F832E83812F902FD8
:10BC0000DF91CF911F910F910895FA01AA27283053
:10BC100051F1203181F1E8946F936E7F6E5F7F4F19
:10BC20008F4F9F4FAF4FB1E03ED0B4E03CD0670F95
:10BC3000781F891F9A1FA11D680F791F8A1F911DE8
:10BC4000A11D6A0F711D811D911DA11D20D009F438
:10BC500068943F912AE0269F11243019305D31937A
:10BC6000DEF6CF010895462F4770405D4193B3E063
:10BC70000FD0C9F7F6CF462F4F70405D4A3318F00A
:10BC8000495D31FD4052419302D0A9F7EACFB4E0BB
:10BC9000A6959795879577956795BA95C9F7009773
:10BCA0006105710508959B01AC010A2E0694579514
:10BCB000479537952795BA95C9F7620F731F841F6B
:0ABCC000951FA01D0895F894FFCF12
:10BCCA00010000000422568001030507090E101224
:0EBCDA001416181C1E2F0070066D066A060058
:00000001FF
